:10000000D7EF23F0FFFFFFFF0BC0FAF40AC0F9F4AB
:10001000E9CF42F4EACF43F4E1CF44F4E2CF45F430
:10002000F2A219D0010E1526000E16221722182250
:10003000F2928C88210E0B6EFF0E0A6E0B2E01D0F1
:1000400003D00A2EFED7FAD7600E0A6E0A2EFED70C
:10005000000000008C989EB09E9042C4E9FF43C40B
:10006000EAFF44C4E1FF45C4E2FFFAC40BF0F9C45F
:100070000AF01100280E0401BE6F6E0EBF6F750EE0
:10008000C06F6C0EC16F6C0EC26F290EC36FC46B54
:10009000CC6BCD6BCA6BCB6B0401B9C400F0BAC496
:1000A00001F0BBC402F0010EB927000EBA23BB2336
:1000B00000C0F6FF01C0F7FF02C0F8FF0900F5CF4E
:1000C00000F000C0C7F40052D8B47AEF11F0C75165
:1000D000250A0BE0B7C4E1FFB8C4E2FFC7C4E6FFDE
:1000E000B74BB82BCC4BCD2BD7D7C86BC96BCA6BD2
:1000F000CB6B040123D0CA87010EB927000EBA23A7
:10010000BB235AD0CA81010EB927000EBA23BB23E4
:1001100053D0CA83010EB927000EBA23BB234CD09B
:10012000CB87010EB927000EBA23BB2345D0CA8561
:10013000010EB927000EBA23BB233ED00401B9C477
:10014000F6FFBAC4F7FFBBC4F8FF0900F5CFD8F437
:10015000D8512D0AD0E0B9C4F6FFBAC4F7FFBBC42A
:10016000F8FF0900F5CFD8F4D851200ACBE0B9C484
:10017000F6FFBAC4F7FFBBC4F8FF0900F5CFD8F407
:10018000D8512B0AC6E0B9C4F6FFBAC4F7FFBBC406
:10019000F8FF0900F5CFD8F4D851230AC1E0B9C45B
:1001A000F6FFBAC4F7FFBBC4F8FF0900F5CFD8F4D7
:1001B000D851300ABCE001D09CD70401CAB3CA911F
:1001C000CAB7CA95B9C4F6FFBAC4F7FFBBC4F8FFF3
:1001D0000900F5CF00F0000E016E00C0E0F4EDEC78
:1001E0003DF0005238E00401C86BC96BC8C400F090
:1001F000C9C401F00A0E046E000E056EDCEC39F085
:10020000B9C4F6FFBAC4F7FFBBC4F8FF0900F5CFC5
:10021000D8F40401D8510024C86F000E0120C96F22
:10022000300EC85F000EC95B010EB927000EBA235D
:10023000BB23B9C4F6FFBAC4F7FFBBC4F8FF09007B
:10024000F5CF00F0000E016E00C0E0F4EDEC3DF0E3
:100250000052CCE136D0B9C4F6FFBAC4F7FFBBC434
:10026000F8FF0900F5CFD8F40401D8512A0A29E192
:10027000BCC4E9FFBDC4EAFFEECF00F0EECF01F051
:1002800000C0E9FF01C0EAFFEECFC8F4EECFC9F429
:10029000BCC4E9FFBDC4EAFFEECF00F0EECF01F031
:1002A000020E0026000E0122BCC4E1FFBDC4E2FF25
:1002B00000C0E6FF01C0E6FF010EB927000EBA2319
:1002C000BB230401B9C4F6FFBAC4F7FFBBC4F8FFEF
:1002D0000900F5CFD8F4D8512E0A74E1010EB927E0
:1002E000000EBA23BB23B9C4F6FFBAC4F7FFBBC4E0
:1002F000F8FF0900F5CFD8F4D8512A0A2AE1BCC486
:10030000E9FFBDC4EAFFEECF00F0EECF01F000C080
:10031000E9FF01C0EAFFEECFC5F4EECFC6F4BCC4DE
:10032000E9FFBDC4EAFFEECF00F0EECF01F0020E10
:100330000026000E0122BCC4E1FFBDC4E2FF00C0E4
:10034000E6FF01C0E6FF010EB927000EBA23BB236A
:1003500037D0C56BC66BB9C4F6FFBAC4F7FFBBC4D0
:10036000F8FF0900F5CF00F0000E016E00C0E0F4C8
:10037000EDEC3DF0005224E0C5C400F0C6C401F02D
:100380000A0E046E000E056EDCEC39F0B9C4F6FFFF
:10039000BAC4F7FFBBC4F8FF0900F5CFD8F40401D5
:1003A000D8510024C56F000E0120C66F300EC55F06
:1003B000000EC65B010EB927000EBA23BB23CBD7B4
:1003C000040104D00401C56BC66BCB890401B9C418
:1003D00000F0BAC401F0BBC402F0010EB927000E50
:1003E000BA23BB2300C0F6FF01C0F7FF02C0F8FF2D
:1003F0000900F5CFC7F4EDD0CCC400F0CDC401F0B6
:100400001200CA89E3D7CB851FD1CA8BCB811CD1FF
:10041000CB831AD1CA8D18D117D1CA8BCA8F14D1E8
:10042000BCC4E9FFBDC4EAFFEECF00F0EECF01F09F
:1004300000C0E9FF01C0EAFFEECFD4F4EECFD5F45F
:10044000BCC4E9FFBDC4EAFFEECF00F0EECF01F07F
:10045000020E0026000E0122BCC4E1FFBDC4E2FF73
:1004600000C0E6FF01C0E6FF000ED51902E1000E54
:10047000D41904E1BE0ED46F040ED56F0401D66BFF
:10048000D76BD651D425E96ED751D521EA6EEECF80
:1004900000F0005203E0D64BD72BF3D7C551C6115D
:1004A0000AE0D751C65D02E1D651C55D04E2C5C47C
:1004B000D6F4C6C4D7F40401C951D75D02E1C851CE
:1004C000D65D05E2D651C85FD751C95B03D00401A0
:1004D000C86BC96BCAB716D0C8C400F0C9C401F054
:1004E000010EC85F000EC95B005001100BE0B7C4DD
:1004F000E1FFB8C4E2FF200EE66EB74BB82BCC4B41
:10050000CD2BEAD7D6C400F0D7C401F0010ED65FD8
:10051000000ED75B0050011013E0D4C4E9FFD5C42E
:10052000EAFFEECF00F0B7C4E1FFB8C4E2FF00C0BD
:10053000E6FFB74BB82BD44BD52BCC4BCD2BE2D70A
:10054000CAA716D0C8C400F0C9C401F0010EC85F24
:10055000000EC95B005001100BE0B7C4E1FFB8C446
:10056000E2FF200EE66EB74BB82BCC4BCD2BEAD773
:1005700093D5BCC4E9FFBDC4EAFFEECF00F0EECFD7
:1005800001F000C0E9FF01C0EAFFEECFC7F4BCC430
:10059000E9FFBDC4EAFFEECF00F0EECF01F0020E9E
:1005A0000026000E0122BCC4E1FFBDC4E2FF00C072
:1005B000E6FF01C0E6FFC70ED46F040ED56F010E33
:1005C000D66F000ED76F6AD7C00ECA13000ECB13BA
:1005D0003BD0C751000AD8B40FD7C7516C0AD8B462
:1005E00010D7C751660AD8B40ED7C751450AD8B438
:1005F0000CD7C751650AD8B409D7C751670AD8B410
:1006000007D7C7516F0AD8B405D7C751640AD8B401
:1006100003D7C751690AD8B4FFD6C751700AD8B4F6
:10062000FCD6C751580AD8B4F8D6C751780AD8B4FE
:10063000F5D6C751730AD8B4F3D6C751630A99E007
:10064000C751750AC1E0B7D70401000ECA15006E84
:10065000CB51070B016E00500110D8B4B0EF0CF075
:10066000CBA904D0060EC56F000EC66FBCC4E9FF4F
:10067000BDC4EAFFEECF00F0EECF01F000C0E9FF0D
:1006800001C0EAFFEECFCEF4EECFCFF4EECFD0F440
:10069000EECFD1F4BCC4E9FFBDC4EAFFEECF00F059
:1006A000EECF01F0040E0026000E0122BCC4E1FFD3
:1006B000BDC4E2FF00C0E6FF01C0E6FF046A056AB0
:1006C000066A076ACEC400F0CFC401F0D0C402F0BD
:1006D000D1C403F0ADEC2FF0010ED8B0000E006EC7
:1006E000005206E00401D07F030ECA13000ECB13A4
:1006F0000401D26BD36BCEC400F0CFC401F0D0C4E0
:1007000002F0D1C403F0046A056A066A076AEDECD8
:100710003CF0000ED8A4010E006E0052D8B49AD05E
:10072000D1C400F0016A026A036AFF0E00140401DA
:10073000DC6F000EDD6F000EDD177E0ED86F000E31
:10074000D96FDA6FDB6FD851DC5D006ED951DD599E
:10075000016E00C0D2F401C0D3F4010E005CD26F70
:10076000000E0158D36FD2C400F0D3C401F0030EC1
:10077000046E000E056EDCEC39F000C0D2F401C04E
:10078000D3F40A0E046E000E056E15EC30F000C0B6
:10079000D2F401C0D3F4800E01180401D86F800E8A
:1007A000D85D02E1000E005C04E2010ED25F000E93
:1007B000D35B0401D2510008E06F23EC15F0CEC4E6
:1007C00004F0CFC405F0D0C406F0D1C407F099EC12
:1007D0002EF000C0D4F401C0D5F402C0D6F403C09A
:1007E000D7F4000E046E000E056E000E066E7F0E2E
:1007F000076ED4C400F0D5C401F0D6C402F0D7C44B
:1008000003F0ADEC2FF0010ED8B0000E006E0052D8
:1008100006E0010E0401D25F000ED35B1BD0000E78
:10082000046E000E056E200E066E820E076ED4C496
:1008300000F0D5C401F0D6C402F0D7C403F0ADEC8B
:100840002FF0000ED8B0010E006E005203E004013C
:10085000D24BD32B0401800E006E800E0401D319FD
:10086000005C02E1D251000803E3010EC76F03D020
:100870000401D2C4C7F4CBB11AD0CBA315D0800EDB
:10088000D319006E7F0E005C02E1FC0ED25D0AE31C
:10089000800ED319006E800EC619005C02E1C551AE
:1008A000D25D02E3040103D004019CEF08F00401CF
:1008B000C551C61106E0CBA304D0010EC55F000EE2
:1008C000C65B000E006EC651005C02E1C55108080F
:1008D00003E2080EC76F03D00401C5C4C7F4CEC439
:1008E00000F0CFC401F0D0C402F0D1C403F0046A18
:1008F000056A066A076AEDEC3CF0000ED8A4010E0A
:10090000006E0052D8B464D1D2C4E0F423EC15F0E8
:1009100000C004F001C005F002C006F003C007F0FB
:10092000CEC400F0CFC401F0D0C402F0D1C403F0B3
:1009300013EC2CF000C0CEF401C0CFF402C0D0F410
:1009400003C0D1F40401C7510008E06F23EC15F097
:1009500000C004F001C005F002C006F003C007F0BB
:10096000CEC400F0CFC401F0D0C402F0D1C403F073
:1009700013EC2CF000C0D8F401C0D9F402C0DAF4B2
:1009800003C0DBF4D8C4CEF4D9C4CFF4DAC4D0F4B5
:10099000DBC4D1F4D8C400F0D9C401F0DAC402F049
:1009A000DBC403F062EC2DF076EC3DF000C004F007
:1009B00001C005F002C006F003C007F0D8C400F083
:1009C000D9C401F0DAC402F0DBC403F08BEC3EF0D2
:1009D000000E046E000E056E000E066E7E0E076E93
:1009E000ADEC2FF0000ED8B0010E006E00521AE0F0
:1009F000CEC400F0CFC401F0D0C402F0D1C403F0E3
:100A0000000E046E000E056E000E066E7E0E076E62
:100A100063EC1AF000C0CEF401C0CFF402C0D0F4F1
:100A200003C0D1F4CEC400F0CFC401F0D0C402F0B2
:100A3000D1C403F062EC2DF000C0DCF401C0DDF4A1
:100A400002C0DEF403C0DFF40401C751010F006EE1
:100A5000016A000E0122020E046E000E01BEFF0E9E
:100A6000026E036E0450040107E000360090013668
:100A700002360336FF0FF7D70401920E00267D0ED3
:100A80000122000E022200C0F6FF01C0F7FF02C0E3
:100A9000F8FF0900F5CFD8F40900F5CFD9F4090023
:100AA000F5CFDAF40900F5CFDBF4DB51DF5D08E1C7
:100AB000DA51DE5D05E1D951DD5D02E1D851DC5D41
:100AC0001EE3CEC400F0CFC401F0D0C402F0D1C404
:100AD00003F0CD0E046ECC0E056E4C0E066E7B0E32
:100AE000076E99EC2EF000C0CEF401C0CFF402C026
:100AF000D0F403C0D1F40401D24BD32B69D004014C
:100B0000CEC400F0CFC401F0D0C402F0D1C403F0D1
:100B100062EC2DF000C0DCF401C0DDF402C0DEF4B4
:100B200003C0DFF4020E046EC7C400F0000E016EB5
:100B3000026E036E0450000107E00036009001369B
:100B400002360336FF0FF7D7920E00267D0E0122E4
:100B5000000E022200C0F6FF01C0F7FF02C0F8FF3E
:100B60000900F5CFD8F40900F5CFD9F40900F5CF85
:100B7000DAF40900F5CFDBF40401DB51DF5D08E1B5
:100B8000DA51DE5D05E1D951DD5D02E1D851DC5D70
:100B90001FE2CEC400F0CFC401F0D0C402F0D1C433
:100BA00003F0000E046E000E056E200E066E820E1F
:100BB000076E99EC2EF000C0CEF401C0CFF402C055
:100BC000D0F403C0D1F4010E0401D25F000ED35B58
:100BD00004010401CBA398D0CBB796D0800E000AB5
:100BE000006E800EC619005C02E1C5510A0804E2DD
:100BF0000A0EC56F000EC66F0401CEC400F0CFC44C
:100C000001F0D0C402F0D1C403F062EC2DF000C0BA
:100C1000D4F401C0D5F402C0D6F403C0D7F4040163
:100C2000D451D511D611D71144E00A0E046E000E2E
:100C3000056E066E076ED4C400F0D5C401F0D6C4AC
:100C400002F0D7C403F0E0EC1FF008C000F009C0C8
:100C500001F00AC002F00BC003F0000E0401D86FCF
:100C6000031808E1D851021805E1D851011802E132
:100C70000050000A1EE1010E0401C55F000EC65BB4
:100C80000A0E046E000E056E066E076ED4C400F0E8
:100C9000D5C401F0D6C402F0D7C403F0E0EC1FF0D5
:100CA00000C0D4F401C0D5F402C0D6F403C0D7F418
:100CB000B6D7800E0401C619006E800E005C02E1FA
:100CC000C751C55D21E2C551C75DE06F23EC15F04A
:100CD00000C004F001C005F002C006F003C007F038
:100CE000CEC400F0CFC401F0D0C402F0D1C403F0F0
:100CF00013EC2CF000C0CEF401C0CFF402C0D0F44D
:100D000003C0D1F4C5C4C7F40001050E0401C52514
:100D1000006E000EC621016E0050C85F0150C95B15
:100D2000C551C61102E1CBA704D0010EC85F000E69
:100D3000C95B030ECA15006ECBC401F0000E01168C
:100D40000050011004E0010EC85F000EC95BCAA587
:100D50004AD0CAA31AD0010ECA15006ECBC401F046
:100D6000000E01160050011003E02D0E006E02D09F
:100D70002B0E006EB7C4E1FFB8C4E2FF00C0E6FF6F
:100D8000B74BB82BCC4BCD2B14D0010ECA15006E2F
:100D9000CBC401F0000E0116005001100AE0B7C4E8
:100DA000E1FFB8C4E2FF200EE66EB74BB82BCC4B88
:100DB000CD2B800E006E800EC919005C02E1C85177
:100DC00000080FE2B7C4E1FFB8C4E2FF300EE66EE0
:100DD000B74BB82BCC4BCD2B010EC85F000EC95BB7
:100DE000E8D704014BD0CAB718D0800E006E800E31
:100DF000C919005C02E1C85100080FE2B7C4E1FF65
:100E0000B8C4E2FF200EE66EB74BB82BCC4BCD2B0F
:100E1000010EC85F000EC95BE8D70401CAA31AD04F
:100E2000010ECA15006ECBC401F0000E0116005071
:100E3000011003E02D0E006E02D02B0E006EB7C421
:100E4000E1FFB8C4E2FF00C0E6FFB74BB82BCC4BC4
:100E5000CD2B14D0010ECA15006ECBC401F0000ECC
:100E60000116005001100AE0B7C4E1FFB8C4E2FF68
:100E7000200EE66EB74BB82BCC4BCD2B0401CEC465
:100E800000F0CFC401F0D0C402F0D1C403F062EC92
:100E90002DF000C0D4F401C0D5F402C0D6F403C0D4
:100EA000D7F4020E046EC7C400F0000E016E026E8D
:100EB000036E0450000107E0003600900136023650
:100EC0000336FF0FF7D7920E00267D0E0122000E8B
:100ED000022200C0F6FF01C0F7FF02C0F8FF0900C0
:100EE000F5CF04F00900F5CF05F00900F5CF06F0C5
:100EF0000900F5CF07F0D4C400F0D5C401F0D6C482
:100F000002F0D7C403F0E0EC1FF0300E0026B7C4A7
:100F1000E1FFB8C4E2FF00C0E6FF0401B74BB82B05
:100F2000CC4BCD2BC551C61102E1CBA776D0B7C4AF
:100F3000E1FFB8C4E2FF2E0EE66E0401B74BB82BFA
:100F4000CC4BCD2BC751C55F000EC65BC75353E0DA
:100F5000C707020E046EC7C400F0000E016E026ED9
:100F6000036E0450040107E000360090013602369B
:100F70000336FF0FF7D7920E00267D0E0122000EDA
:100F8000022200C0F6FF01C0F7FF02C0F8FF09000F
:100F9000F5CF04F00900F5CF05F00900F5CF06F014
:100FA0000900F5CF07F0D4C400F0D5C401F0D6C4D1
:100FB00002F0D7C403F0E0EC1FF00A0E046E000E3E
:100FC000056E066E076EE0EC1FF008C000F009C069
:100FD00001F00AC002F00BC003F0300E0026B7C4C7
:100FE000E1FFB8C4E2FF00C0E6FF0401B74BB82B35
:100FF000CC4BCD2BABD7C551C6110FE0B7C4E1FF29
:10100000B8C4E2FF300EE66EB74BB82BCC4BCD2BFD
:10101000010EC55F000EC65BEED7CAAB0BD0B7C4DE
:10102000E1FFB8C4E2FF450EE66EB74BB82BCC4BE0
:10103000CD2B0AD0B7C4E1FFB8C4E2FF650EE66E5F
:10104000B74BB82BCC4BCD2B800ED319006E800E36
:10105000005C02E1000ED25D12E2D2510008D26FB4
:10106000D3C4D3F4E86AD357B7C4E1FFB8C4E2FFEE
:101070002D0EE66EB74BB82BCC4BCD2B0BD004010D
:10108000B7C4E1FFB8C4E2FF2B0EE66EB74BB82B36
:10109000CC4BCD2B0A0E046E000E056ED2C400F0B0
:1010A000D3C401F015EC30F0300E0026B7C4E1FFD8
:1010B000B8C4E2FF00C0E6FF0401B74BB82BCC4B2D
:1010C000CD2B0A0E046E000E056ED2C400F0D3C400
:1010D00001F015EC30F008C000F009C001F0300E4E
:1010E0000026B7C4E1FFB8C4E2FF00C0E6FF040178
:1010F000B74BB82BCC4BCD2BCAA71BD0800E006EA4
:10110000800EC919005C02E1C851000812E2B7C4A0
:10111000E1FFB8C4E2FF200EE66E0401B74BB82B26
:10112000CC4BCD2B010EC85F000EC95BC851C91155
:10113000EEE104014CEF00F00401CBA3FDD0800EE2
:10114000D319006E800E005C02E1000ED25D0AE24F
:10115000010ED25D006E000ED359016E0050C55FC6
:101160000150C65BCEC400F0CFC401F0D0C402F081
:10117000D1C403F062EC2DF000C0D4F401C0D5F46A
:1011800002C0D6F403C0D7F4010E0401C76FC751E3
:101190000A0A39E0020E046EC7C400F0000E016EA8
:1011A000026E036E0450040107E000360090013621
:1011B00002360336FF0FF7D70401920E00267D0E8C
:1011C0000122000E022200C0F6FF01C0F7FF02C09C
:1011D000F8FF0900F5CFD8F40900F5CFD9F40900DC
:1011E000F5CFDAF40900F5CFDBF4DB51D75D08E188
:1011F000DA51D65D05E1D951D55D02E1D851D45D12
:1012000002E3C72BC4D70401C751C55DDC6F000ED4
:10121000C659DD6FDCC4C5F4DDC4C6F4D4C400F027
:10122000D5C401F0D6C402F0D7C403F076EC3DF08B
:1012300000C004F001C005F002C006F003C007F0D2
:10124000CEC400F0CFC401F0D0C402F0D1C403F08A
:101250008BEC3EF000C0D8F401C0D9F402C0DAF43F
:1012600003C0DBF4DCC4E0F423EC15F0D8C404F0D4
:10127000D9C405F0DAC406F0DBC407F099EC2EF00F
:10128000000E046E000E056E000E066E7E0E076EDA
:1012900063EC1AF062EC2DF000C0D4F401C0D5F478
:1012A00002C0D6F403C0D7F40401C551C61144E00E
:1012B0000A0E046E000E056E066E076ED4C400F0B2
:1012C000D5C401F0D6C402F0D7C403F0E0EC1FF09F
:1012D00008C000F009C001F00AC002F00BC003F022
:1012E000000E0401D86F031808E1D851021805E177
:1012F000D851011802E10050000A1EE10A0E046EE6
:10130000000E056E066E076ED4C400F0D5C401F061
:10131000D6C402F0D7C403F0E0EC1FF000C0D4F450
:1013200001C0D5F402C0D6F403C0D7F4010E040105
:10133000C55F000EC65BB8D70401800E006E800E3C
:101340000401C619005C02E1C5510C0816E3C5C4CE
:10135000E0F44DEC1EF0CEC404F0CFC405F0D0C4D0
:1013600006F0D1C407F063EC1AF000C0CEF401C05F
:10137000CFF402C0D0F403C0D1F4CEC400F0CFC487
:1013800001F0D0C402F0D1C403F0046A056A066A11
:10139000076AEDEC3CF0000ED8A4010E006E00527E
:1013A000D8B478D0CEC400F0CFC401F0D0C402F0DD
:1013B000D1C403F062EC2DF0000E0401D86F0318C5
:1013C00008E1D851021805E1D851011802E1005096
:1013D000000A60E1800E006E800ED319005C02E10D
:1013E000D251010857E2D2C4E0F423EC15F000C05A
:1013F00004F001C005F002C006F003C007F0CEC43F
:1014000000F0CFC401F0D0C402F0D1C403F013EC5B
:101410002CF05F0E046E700E056E090E066E810EC6
:10142000076EADEC2FF0010ED8B0000E006E00522A
:1014300006E0090E0401D25F000ED35B05D0080E52
:101440000401D25F000ED35BD2C4E0F423EC15F0AC
:1014500000C004F001C005F002C006F003C007F0B0
:10146000CEC400F0CFC401F0D0C402F0D1C403F068
:1014700013EC2CF062EC2DF000C0D4F401C0D5F4D4
:1014800002C0D6F403C0D7F40401CE6BCF6BD06B8F
:10149000D16B39D0CEC400F0CFC401F0D0C402F07B
:1014A000D1C403F062EC2DF000C0D4F401C0D5F437
:1014B00002C0D6F403C0D7F4D4C400F0D5C401F000
:1014C000D6C402F0D7C403F076EC3DF000C004F0BF
:1014D00001C005F002C006F003C007F0CEC400F062
:1014E000CFC401F0D0C402F0D1C403F08BEC3EF0C5
:1014F00000C0CEF401C0CFF402C0D0F403C0D1F4D8
:101500000401D26BD36B010EC76FC7510A0A39E0D1
:10151000020E046EC7C400F0000E016E026E036E70
:101520000450040107E0003600900136023603360D
:10153000FF0FF7D70401920E00267D0E0122000E48
:10154000022200C0F6FF01C0F7FF02C0F8FF090049
:10155000F5CFD8F40900F5CFD9F40900F5CFDAF4C6
:101560000900F5CFDBF4DB51D75D08E1DA51D65D38
:1015700005E1D951D55D02E1D851D45D02E3C72B15
:10158000C4D70401C751C525006E000EC621016EE7
:10159000D2510026D35101220050C85F0150C95BCF
:1015A000CBB703D0C551C61104E0010EC85F000ED1
:1015B000C95B030ECA15006ECBC401F0000E011604
:1015C0000050011004E0010EC85F000EC95BCAA5FF
:1015D0004AD0CAA31AD0010ECA15006ECBC401F0BE
:1015E000000E01160050011003E02D0E006E02D017
:1015F0002B0E006EB7C4E1FFB8C4E2FF00C0E6FFE7
:10160000B74BB82BCC4BCD2B14D0010ECA15006EA6
:10161000CBC401F0000E0116005001100AE0B7C45F
:10162000E1FFB8C4E2FF200EE66EB74BB82BCC4BFF
:10163000CD2B800E006E800EC919005C02E1C851EE
:1016400000080FE2B7C4E1FFB8C4E2FF300EE66E57
:10165000B74BB82BCC4BCD2B010EC85F000EC95B2E
:10166000E8D704014BD0CAB718D0800E006E800EA8
:10167000C919005C02E1C85100080FE2B7C4E1FFDC
:10168000B8C4E2FF200EE66EB74BB82BCC4BCD2B87
:10169000010EC85F000EC95BE8D70401CAA31AD0C7
:1016A000010ECA15006ECBC401F0000E01160050E9
:1016B000011003E02D0E006E02D02B0E006EB7C499
:1016C000E1FFB8C4E2FF00C0E6FFB74BB82BCC4B3C
:1016D000CD2B14D0010ECA15006ECBC401F0000E44
:1016E0000116005001100AE0B7C4E1FFB8C4E2FFE0
:1016F000200EE66EB74BB82BCC4BCD2B0401C7C4E4
:1017000000F0C707005252E0020E046EC7C400F09A
:10171000000E016E026E036E0450040107E00036F5
:101720000090013602360336FF0FF7D7920E0026DF
:101730007D0E0122000E022200C0F6FF01C0F7FF5D
:1017400002C0F8FF0900F5CF04F00900F5CF05F05D
:101750000900F5CF06F00900F5CF07F0D4C400F07A
:10176000D5C401F0D6C402F0D7C403F0E0EC1FF0FA
:101770000A0E046E000E056E066E076EE0EC1FF09A
:1017800008C000F009C001F00AC002F00BC003F06D
:10179000300E0026B7C4E1FFB8C4E2FF00C0E6FF88
:1017A0000401B74BB82BCC4BCD2BA8D7800E006EC5
:1017B000800ED319005C02E1D25100080FE2B7C4D9
:1017C000E1FFB8C4E2FF300EE66EB74BB82BCC4B4E
:1017D000CD2B010ED25F000ED35BE8D70401800E43
:1017E000000A006E800EC619005C02E1C5510808AF
:1017F00003E2080EC76F03D00401C5C4C7F4C75184
:10180000C55F000EC65BC75302E1CBA70AD0B7C4C1
:10181000E1FFB8C4E2FF2E0EE66EB74BB82BCC4BFF
:10182000CD2BC7C4E0F423EC15F0CEC404F0CFC434
:1018300005F0D0C406F0D1C407F099EC2EF0FFEC0F
:101840002DF000C0D4F401C0D5F402C0D6F403C01A
:10185000D7F40401C75353E0C707020E046EC7C490
:1018600000F0000E016E026E036E0450040107E0EA
:1018700000360090013602360336FF0FF7D7920E7E
:1018800000267D0E0122000E022200C0F6FF01C0DC
:10189000F7FF02C0F8FF0900F5CF04F00900F5CF0B
:1018A00005F00900F5CF06F00900F5CF07F0D4C424
:1018B00000F0D5C401F0D6C402F0D7C403F0E0ECC8
:1018C0001FF00A0E046E000E056E066E076EE0EC49
:1018D0001FF008C000F009C001F00AC002F00BC000
:1018E00003F0300E0026B7C4E1FFB8C4E2FF00C029
:1018F000E6FF0401B74BB82BCC4BCD2BAAD7C55173
:10190000C6110FE0B7C4E1FFB8C4E2FF300EE66EC7
:10191000B74BB82BCC4BCD2B010EC55F000EC65B71
:10192000EED7CAA71AD0800E006E800EC919005CCF
:1019300002E1C851000811E2B7C4E1FFB8C4E2FFF8
:10194000200EE66EB74BB82BCC4BCD2B010EC85FEB
:10195000000EC95BC851C911EFE104014CEF00F062
:10196000C00ECA15D86FCBC4D9F4000ED917000E1B
:10197000D91902E1000ED819D8A482D0CAA929D059
:10198000BCC4E9FFBDC4EAFFEECF00F0EECF01F02A
:1019900000C0E9FF01C0EAFFEECFD4F4EECFD5F4EA
:1019A000EECFD6F4EECFD7F4BCC4E9FFBDC4EAFF56
:1019B000EECF00F0EECF01F0040E0026000E012263
:1019C000BCC4E1FFBDC4E2FF00C0E6FF01C0E6FF0A
:1019D0002ED0BCC4E9FFBDC4EAFFEECF00F0EECFCD
:1019E00001F000C0E9FF01C0EAFFEECFD4F4EECF72
:1019F000D5F4000ED5BFFF0ED66FD76F000ED5BF42
:101A0000FF0ED66FD76FBCC4E9FFBDC4EAFFEECFAF
:101A100000F0EECF01F0020E0026000E0122BCC441
:101A2000E1FFBDC4E2FF00C0E6FF01C0E6FF800E9B
:101A3000D719006E800E005C08E1000ED65D05E14E
:101A4000000ED55D02E1000ED45D18E2030ECA134C
:101A5000000ECB13006A016A026A036AD451005E69
:101A6000D551015AD651025AD751035A00C0D4F465
:101A700001C0D5F402C0D6F403C0D7F4040156D097
:101A80000401CAA929D0BCC4E9FFBDC4EAFFEECF56
:101A900000F0EECF01F000C0E9FF01C0EAFFEECF99
:101AA000D4F4EECFD5F4EECFD6F4EECFD7F4BCC459
:101AB000E9FFBDC4EAFFEECF00F0EECF01F0040E67
:101AC0000026000E0122BCC4E1FFBDC4E2FF00C03D
:101AD000E6FF01C0E6FF2AD0BCC4E9FFBDC4EAFFAF
:101AE000EECF00F0EECF01F000C0E9FF01C0EAFF49
:101AF000EECFD4F4EECFD5F4000ED66FD76F000E34
:101B0000D66FD76FBCC4E9FFBDC4EAFFEECF00F0CB
:101B1000EECF01F0020E0026000E0122BCC4E1FF50
:101B2000BDC4E2FF00C0E6FF01C0E6FF0401000EF5
:101B3000C61902E1000EC5190FE1000E006ED7199B
:101B400008E10050D61905E10050D51902E1D45141
:101B5000000A02E1C54BC62B0401C00ECA15006E77
:101B600000C0DCF4C0D0010EC76FC7510A0A39E0CB
:101B7000020E046EC7C400F0000E016E026E036E0A
:101B80000450040107E000360090013602360336A7
:101B9000FF0FF7D70401920E00267D0E0122000EE2
:101BA000022200C0F6FF01C0F7FF02C0F8FF0900E3
:101BB000F5CFD8F40900F5CFD9F40900F5CFDAF460
:101BC0000900F5CFDBF4DB51D75D08E1DA51D65DD2
:101BD00005E1D951D55D02E1D851D45D02E3C72BAF
:101BE000C4D704018FD0010EC76FC751080A39E06E
:101BF000020E046EC7C400F0000E016E026E036E8A
:101C00000450040107E00036009001360236033626
:101C1000FF0FF7D70401BA0E00267D0E0122000E39
:101C2000022200C0F6FF01C0F7FF02C0F8FF090062
:101C3000F5CFD8F40900F5CFD9F40900F5CFDAF4DF
:101C40000900F5CFDBF4DB51D75D08E1DA51D65D51
:101C500005E1D951D55D02E1D851D45D02E3C72B2E
:101C6000C4D704014FD0010EC76FC7510C0A39E029
:101C7000020E046EC7C400F0000E016E026E036E09
:101C80000450040107E000360090013602360336A6
:101C9000FF0FF7D70401DA0E00267D0E0122000E99
:101CA000022200C0F6FF01C0F7FF02C0F8FF0900E2
:101CB000F5CFD8F40900F5CFD9F40900F5CFDAF45F
:101CC0000900F5CFDBF4DB51D75D08E1DA51D65DD1
:101CD00005E1D951D55D02E1D851D45D02E3C72BAE
:101CE000C4D704010FD0DC51000AD8B43CD7DC5172
:101CF000C00AD8B438D7DC51800AD8B474D7DC51C4
:101D0000400AB1E00401800E006E800EC619005C2E
:101D100002E1C551C75D03E2C5C4C7F40ED004019A
:101D2000800EC619006E800E005C02E1C751C55DD1
:101D300004E2C7C4C5F4000EC66F04010401C85113
:101D4000C9110EE0030ECA15006ECBC401F0000EDF
:101D500001160050011004E0010EC85F000EC95BBF
:101D6000800EC619006E800EC919005C02E1C851D0
:101D7000C55D05E2C551C85FC651C95B03D004010A
:101D8000C86BC96BC40ECA15D86FCB51080BD96F7D
:101D9000D951080A02E1400ED81908E1C851C91109
:101DA00004E0010EC85F000EC95B1ED00401C00E26
:101DB000CA15D86FCB51080BD96FD951080A02E167
:101DC000800ED81911E1800E006E800EC919005CDA
:101DD00002E1C851020805E2020EC85F000EC95BAD
:101DE00003D00401C86BC96B04010401CAA56ED0FD
:101DF000CAA31AD0010ECA15006ECBC401F0000EA2
:101E000001160050011003E02D0E006E02D02B0EC3
:101E1000006EB7C4E1FFB8C4E2FF00C0E6FFB74BF5
:101E2000B82BCC4BCD2B3CD0010ECA15006ECBC4C9
:101E300001F0000E0116005001100BE0B7C4E1FFE5
:101E4000B8C4E2FF200EE66EB74BB82BCC4BCD2BBF
:101E500027D0C00ECA15D86FCB51080BD96FD951F6
:101E6000080A02E1800ED8191BE1B7C4E1FFB8C42B
:101E7000E2FF300EE66EB74BB82BCC4BCD2BCAAB86
:101E800003D0580E006E02D0780E006EB7C4E1FF8A
:101E9000B8C4E2FF00C0E6FFB74BB82BCC4BCD2B4C
:101EA0000401C851C91111E0B7C4E1FFB8C4E2FF91
:101EB000300EE66EB74BB82BCC4BCD2B010EC85F66
:101EC000000EC95BC851C911EFE185D0C851C911D5
:101ED00013E0CAB711D0B7C4E1FFB8C4E2FF200EC7
:101EE000E66EB74BB82BCC4BCD2B010EC85F000E66
:101EF000C95BC851C911EFE1CAA31AD0010ECA15B6
:101F0000006ECBC401F0000E01160050011003E07A
:101F10002D0E006E02D02B0E006EB7C4E1FFB8C4C8
:101F2000E2FF00C0E6FFB74BB82BCC4BCD2B14D053
:101F3000010ECA15006ECBC401F0000E0116005050
:101F400001100AE0B7C4E1FFB8C4E2FF200EE66E5C
:101F5000B74BB82BCC4BCD2BC00ECA15D86FCB517D
:101F6000080BD96FD951080A02E1400ED8190BE1CC
:101F7000B7C4E1FFB8C4E2FF300EE66EB74BB82B32
:101F8000CC4BCD2B28D00401C00ECA15D86FCB5135
:101F9000080BD96FD951080A02E1800ED8191BE14C
:101FA000B7C4E1FFB8C4E2FF300EE66EB74BB82B02
:101FB000CC4BCD2BCAAB03D0580E006E02D0780E9E
:101FC000006EB7C4E1FFB8C4E2FF00C0E6FFB74B44
:101FD000B82BCC4BCD2B04010401800E006E800E7B
:101FE000C619005C02E1C551C75D0BE2B7C4E1FF51
:101FF000B8C4E2FF300EE66EB74BB82BCC4BCD2BFE
:10200000EAD70401C5C400F0C6C401F0010EC55FE3
:10201000000EC65B00500110D8B44DD1C00ECA15D9
:10202000006E00C0D8F42BD1020E046EC5C400F0BF
:10203000C6C401F0000EC6BFFF0E026E036E045050
:10204000040107E000360090013602360336FF0F28
:10205000F7D7920E00267D0E0122000E022200C04C
:10206000F6FF01C0F7FF02C0F8FF0900F5CF04F04A
:102070000900F5CF05F00900F5CF06F00900F5CF0E
:1020800007F0D4C400F0D5C401F0D6C402F0D7C420
:1020900003F0E0EC1FF00A0E046E000E056E066EF3
:1020A000076EE0EC1FF008C000F009C001F00AC0A4
:1020B00002F00BC003F0300E00240401C76FEFD014
:1020C000CAAB4ED0020E046EC5C400F0C6C401F007
:1020D000000EC6BFFF0E026E036E0450040107E03F
:1020E00000360090013602360336FF0FF7D70401A1
:1020F000BA0E00267D0E0122000E022200C0F6FF5D
:1021000001C0F7FF02C0F8FF0900F5CF04F0090095
:10211000F5CF05F00900F5CF06F00900F5CF07F07F
:10212000D4C400F0D5C401F0D6C402F0D7C403F083
:10213000E0EC1FF00F0E0016000E0116021603163B
:102140000A0E00267E0E0122000E022200C0F6FFBB
:1021500001C0F7FF02C0F8FF0900F5CFC7F44ED069
:10216000020E046EC5C400F0C6C401F0000E0401E6
:10217000C6BFFF0E026E036E0450040107E0003676
:102180000090013602360336FF0FF7D70401BA0E6E
:1021900000267D0E0122000E022200C0F6FF01C0C3
:1021A000F7FF02C0F8FF0900F5CF04F00900F5CFF2
:1021B00005F00900F5CF06F00900F5CF07F0D4C40B
:1021C00000F0D5C401F0D6C402F0D7C403F0E0ECAF
:1021D0001FF00F0E0016000E0116021603161C0E3D
:1021E00000267E0E0122000E022200C0F6FF01C072
:1021F000F7FF02C0F8FF0900F5CFC7F400014FD088
:10220000020E046EC5C400F0C6C401F0000E040145
:10221000C6BFFF0E026E036E0450040107E00036D5
:102220000090013602360336FF0FF7D7DA0E00268C
:102230007D0E0122000E022200C0F6FF01C0F7FF52
:1022400002C0F8FF0900F5CF04F00900F5CF05F052
:102250000900F5CF06F00900F5CF07F0D4C400F06F
:10226000D5C401F0D6C402F0D7C403F0E0EC1FF0EF
:10227000070E00140401C76F300EC72710D00401E9
:10228000D851000AD8B4D0D6D851C00AD8B4CCD6C8
:10229000D851800AD8B414D7D851400AB1E004010B
:1022A000B7C4E1FFB8C4E2FFC7C4E6FFB74BB82B21
:1022B000CC4BCD2BA6D6CAA71AD0800E006E800EAE
:1022C000C919005C02E1C851000811E2B7C4E1FF7E
:1022D000B8C4E2FF200EE66EB74BB82BCC4BCD2B2B
:1022E000010EC85F000EC95BC851C911EFE10401BE
:1022F0004CEF00F0CCC400F0CDC401F0120002019C
:10230000FF53D8B49FD3FF6B1EEC26F032C300F00E
:1023100033C301F034C302F035C303F076EC3DF073
:10232000520E046EB80E056E1E0E066E6B0E076E14
:1023300099EC2EF000C078F401C079F402C07AF470
:1023400003C07BF478C412F479C413F47AC414F48F
:102350007BC415F436C300F037C301F038C302F074
:1023600039C303F076EC3DF0520E046EB80E056EE4
:102370001E0E066E6B0E076E99EC2EF000C074F404
:1023800001C075F402C076F403C077F474C416F487
:1023900075C417F476C418F477C419F43AC300F07E
:1023A0003BC301F03CC302F03DC303F076EC3DF0CB
:1023B000520E046EB80E056E1E0E066E6B0E076E84
:1023C00099EC2EF000C070F401C071F402C072F4F8
:1023D00003C073F470C41AF471C41BF472C41CF407
:1023E00073C41DF43EC300F03FC301F040C302F0CC
:1023F00041C303F076EC3DF0520E046EB80E056E4C
:102400001E0E066E6B0E076E99EC2EF000C06CF47B
:1024100001C06DF402C06EF403C06FF46CC41EF40E
:102420006DC41FF46EC420F46FC421F442C300F0E5
:1024300043C301F044C302F045C303F076EC3DF022
:10244000520E046EB80E056E1E0E066E6B0E076EF3
:1024500099EC2EF000C068F401C069F402C06AF47F
:1024600003C06BF468C422F469C423F46AC424F47E
:102470006BC425F446C300F047C301F048C302F023
:1024800049C303F076EC3DF0520E046EB80E056EB3
:102490001E0E066E6B0E076E99EC2EF000C064F4F3
:1024A00001C065F402C066F403C067F464C426F496
:1024B00065C427F466C428F467C429F44AC300F04D
:1024C0004BC301F04CC302F04DC303F076EC3DF07A
:1024D000520E046EB80E056E1E0E066E6B0E076E63
:1024E00099EC2EF000C060F401C061F402C062F407
:1024F00003C063F460C42AF461C42BF462C42CF4F6
:1025000063C42DF42EC300F02FC301F030C302F0DA
:1025100031C303F076EC3DF0520E046EB80E056E3A
:102520001E0E066E6B0E076E99EC2EF000C05CF46A
:1025300001C05DF402C05EF403C05FF45CC42EF41D
:102540005DC42FF45EC430F45FC431F4170E046E22
:10255000B70E056E510E066E710E076E78C400F050
:1025600079C401F07AC402F07BC403F08BEC3EF036
:1025700000C012F401C013F402C014F403C015F437
:10258000170E046EB70E056E510E066E710E076EB5
:1025900074C400F075C401F076C402F077C403F08F
:1025A0008BEC3EF000C016F401C017F402C018F422
:1025B00003C019F4170E046EB70E056E510E066EA9
:1025C000710E076E70C400F071C401F072C402F0A5
:1025D00073C403F08BEC3EF000C01AF401C01BF48E
:1025E00002C01CF403C01DF4170E046EB70E056E76
:1025F000510E066E710E076E6CC400F06DC401F0D2
:102600006EC402F06FC403F08BEC3EF000C01EF409
:1026100001C01FF402C020F403C021F4170E046EA1
:10262000B70E056E510E066E710E076E68C400F08F
:1026300069C401F06AC402F06BC403F08BEC3EF095
:1026400000C022F401C023F402C024F403C025F426
:10265000170E046EB70E056E510E066E710E076EE4
:1026600064C400F065C401F066C402F067C403F0FE
:102670008BEC3EF000C026F401C027F402C028F421
:1026800003C029F4170E046EB70E056E510E066EC8
:10269000710E076E60C400F061C401F062C402F004
:1026A00063C403F08BEC3EF000C02AF401C02BF4AD
:1026B00002C02CF403C02DF4170E046EB70E056E85
:1026C000510E066E710E076E5CC400F05DC401F021
:1026D0005EC402F05FC403F08BEC3EF000C02EF449
:1026E00001C02FF402C030F403C031F403C300F082
:1026F00004C301F034EC3DF03E0E046E050E056E91
:10270000420E066E800E076E99EC2EF0330E046EAC
:10271000330E056E530E066E760E076E99EC2EF094
:1027200000C032F401C033F402C034F403C035F405
:1027300005C300F006C301F034EC3DF03E0E046E1C
:10274000050E056E420E066E800E076E99EC2EF099
:10275000330E046E330E056E530E066E760E076E44
:1027600099EC2EF000C036F401C037F402C038F402
:1027700003C039F407C300F008C301F034EC3DF0A6
:102780003E0E046E050E056E420E066E800E076E3E
:1027900099EC2EF0330E046E330E056E530E066E5A
:1027A000760E076E99EC2EF000C03AF401C03BF4AF
:1027B00002C03CF403C03DF409C300F00AC301F0B9
:1027C00034EC3DF03E0E046E050E056E420E066EB4
:1027D000800E076E99EC2EF0330E046E330E056EEC
:1027E000530E066E760E076E99EC2EF000C03EF486
:1027F00001C03FF402C040F403C041F45CEC32F08D
:102800004EC300F04FC301F03C0E046E000E056E87
:10281000DCEC39F003015051002651510122E5EC66
:102820003BF0000E046E000E056E340E066E890E2F
:10283000076E13EC2CF000C05CF401C05DF402C024
:102840005EF403C05FF452C300F053C301F0E5EC43
:102850003BF05CC404F05DC405F05EC406F05FC4E8
:1028600007F063EC1AF08C887D0E04017C6F030E78
:102870007D6F2E0E7E6F7E0E7F6F000E806F0DC4FB
:1028800081F40EC482F40FC483F410C484F452C3E0
:1028900085F453C386F454C387F455C388F456C3F0
:1028A00089F457C38AF44EC38BF44FC38CF450C3DE
:1028B0008DF451C38EF400C08FF401C090F402C0B7
:1028C00091F403C092F412C493F413C494F414C4A6
:1028D00095F415C496F416C497F417C498F418C464
:1028E00099F419C49AF41AC49BF41BC49CF41CC434
:1028F0009DF41DC49EF41EC49FF41FC4A0F420C404
:10290000A1F421C4A2F422C4A3F423C4A4F424C4D3
:10291000A5F425C4A6F426C4A7F427C4A8F428C4A3
:10292000A9F429C4AAF42AC4ABF42BC4ACF42CC473
:10293000ADF42DC4AEF42EC4AFF42FC4B0F430C443
:10294000B1F431C4B2F452EC3BF0010E0D27000E8D
:102950000E230F2310237D0E7C6F030E7D6FBAECC8
:102960003CF000C07EF401C07FF47D0E7C6F030E4E
:102970007D6F20EC27F07D0E04017C6F030E7D6FD0
:1029800028EC3CF07D0E04017C6F030E7D6F7E0E03
:102990007E6F7E0E7F6F000E806F32C481F433C471
:1029A00082F434C483F435C484F436C485F437C463
:1029B00086F438C487F439C488F43AC489F43BC433
:1029C0008AF43CC48BF43DC48CF43EC48DF43FC403
:1029D0008EF440C48FF441C490F40BC391F40CC343
:1029E00092F40DC393F40EC394F40FC395F410C383
:1029F00096F415C097F416C098F417C099F418C04F
:102A00009AF40BC49BF40CC49CF452EC3BF01EEC07
:102A100026F07D0E04017C6F030E7D6FBAEC3CF056
:102A200000C07EF401C07FF47D0E7C6F030E7D6FCD
:102A300020EC27F07D0E04017C6F030E7D6F28ECE7
:102A40003CF08C981200800E0401E019006E800E9C
:102A5000000A005CD8B081D1E0510008046E04C0C7
:102A6000E0F4800E0418006E800E6E0A005CD8A0A0
:102A7000C6D0640E046EE0C400F001EC32F0120E19
:102A80000026000E00BEFF0E016E000E0122020E97
:102A9000046E000E01BEFF0E026E036E04500001B4
:102AA00007E000360090013602360336FF0FF7D7F5
:102AB00000012A0E00267D0E0122000E022200C017
:102AC000F6FF01C0F7FF02C0F8FF0900F5CFE1F4FF
:102AD0000900F5CFE2F40900F5CFE3F40900F5CFE2
:102AE000E4F4640E046EE0C400F001EC32F008C0BF
:102AF00000F00A0E046E01EC32F0090E0026000E02
:102B000000BEFF0E016E000E0122020E046E000ECA
:102B100001BEFF0E026E036E0450000107E0003696
:102B20000090013602360336FF0FF7D700012A0E58
:102B300000267D0E0122000E022200C0F6FF01C019
:102B4000F7FF02C0F8FF0900F5CF00F00900F5CF4C
:102B500001F00900F5CF02F00900F5CF03F0E1C460
:102B600004F0E2C405F0E3C406F0E4C407F099EC15
:102B70002EF000C0E1F401C0E2F402C0E3F403C0AF
:102B8000E4F40A0E046EE0C400F001EC32F008C078
:102B900000F0020E046E000E00BEFF0E016E026E0B
:102BA000036E0450000107E0003600900136023643
:102BB0000336FF0FF7D700012A0E00267D0E0122F3
:102BC000000E022200C0F6FF01C0F7FF02C0F8FFAE
:102BD0000900F5CF00F00900F5CF01F00900F5CFAD
:102BE00002F00900F5CF03F0E1C404F0E2C405F0FF
:102BF000E3C406F0E4C407F099EC2EF01200800E56
:102C00000A0A006E800E0401E019005C76E20A0EEA
:102C1000046EE0C400F001EC32F0090E0026000E54
:102C200000BEFF0E016E000E0122020E046E000EA9
:102C300001BEFF0E026E036E0450000107E0003675
:102C40000090013602360336FF0FF7D700012A0E37
:102C500000267D0E0122000E022200C0F6FF01C0F8
:102C6000F7FF02C0F8FF0900F5CFE1F40900F5CF46
:102C7000E2F40900F5CFE3F40900F5CFE4F40A0E1D
:102C8000046EE0C400F001EC32F008C000F0020E67
:102C9000046E000E00BEFF0E016E026E036E045045
:102CA000000107E000360090013602360336FF0FC0
:102CB000F7D700012A0E00267D0E0122000E022207
:102CC00000C0F6FF01C0F7FF02C0F8FF0900F5CF12
:102CD00000F00900F5CF01F00900F5CF02F009007E
:102CE000F5CF03F0E1C404F0E2C405F0E3C406F05C
:102CF000E4C407F099EC2EF012000001020E046EFD
:102D0000E0C400F0000E0401E0BFFF0E016E026E91
:102D1000036E0450040107E00036009001360236CD
:102D20000336FF0FF7D704012A0E00267D0E01227D
:102D3000000E022200C0F6FF01C0F7FF02C0F8FF3C
:102D40000900F5CF00F00900F5CF01F00900F5CF3B
:102D500002F00900F5CF03F01200800EE019006EBA
:102D6000800E6E0A005CD8A0C6D0640E046EE0C46B
:102D700000F001EC32F0120E0026000E00BEFF0E35
:102D8000016E000E0122020E046E000E01BEFF0E47
:102D9000026E036E0450000107E000360090013619
:102DA00002360336FF0FF7D700015E0E00267D0EB8
:102DB0000122000E022200C0F6FF01C0F7FF02C090
:102DC000F8FF0900F5CFE1F40900F5CFE2F40900BE
:102DD000F5CFE3F40900F5CFE4F4640E046EE0C42B
:102DE00000F001EC32F008C000F00A0E046E01ECB5
:102DF00032F0090E0026000E00BEFF0E016E000E1E
:102E00000122020E046E000E01BEFF0E026E036E62
:102E10000450000107E00036009001360236033608
:102E2000FF0FF7D700015E0E00267D0E0122000E77
:102E3000022200C0F6FF01C0F7FF02C0F8FF090040
:102E4000F5CF00F00900F5CF01F00900F5CF02F051
:102E50000900F5CF03F0E1C404F0E2C405F0E3C4D7
:102E600006F0E4C407F099EC2EF000C0E1F401C0D4
:102E7000E2F402C0E3F403C0E4F40A0E046EE0C41A
:102E800000F001EC32F008C000F0020E046E000EFB
:102E900000BEFF0E016E026E036E0450000107E0DB
:102EA00000360090013602360336FF0FF7D70001D7
:102EB0005E0E00267D0E0122000E022200C0F6FFEB
:102EC00001C0F7FF02C0F8FF0900F5CF00F00900CC
:102ED000F5CF01F00900F5CF02F00900F5CF03F0BE
:102EE000E1C404F0E2C405F0E3C406F0E4C407F072
:102EF00099EC2EF01200800E0A0A006E800E04017A
:102F0000E019005C76E20A0E046EE0C400F001EC09
:102F100032F0090E0026000E00BEFF0E016E000EFC
:102F20000122020E046E000E01BEFF0E026E036E41
:102F30000450000107E000360090013602360336E7
:102F4000FF0FF7D700015E0E00267D0E0122000E56
:102F5000022200C0F6FF01C0F7FF02C0F8FF09001F
:102F6000F5CFE1F40900F5CFE2F40900F5CFE3F481
:102F70000900F5CFE4F40A0E046EE0C400F001ECA1
:102F800032F008C000F0020E046E000E00BEFF0E0C
:102F9000016E026E036E0450000107E000360090DF
:102FA000013602360336FF0FF7D700015E0E00260A
:102FB0007D0E0122000E022200C0F6FF01C0F7FFC5
:102FC00002C0F8FF0900F5CF00F00900F5CF01F0CD
:102FD0000900F5CF02F00900F5CF03F0E1C404F0D9
:102FE000E2C405F0E3C406F0E4C407F099EC2EF067
:102FF00012000001020E046EE0C400F0000E040195
:10300000E0BFFF0E016E026E036E0450040107E084
:1030100000360090013602360336FF0FF7D75E0EFA
:1030200000267D0E0122000E022200C0F6FF01C024
:10303000F7FF02C0F8FF0900F5CF00F00900F5CF57
:1030400001F00900F5CF02F00900F5CF03F01200FE
:103050000401836B846B7CC4B7F47DC4B8F47EC474
:10306000B9F47AEC30F0842B005203E0320E845D28
:10307000F2E3320E845D03E3FF0E006E12006EEC8D
:1030800038F055C2E5F456C2E6F457C2E7F458C228
:10309000E8F4250E0401E96F000EEA6F69EC33F0E5
:1030A00002012351550AD8A468D02451AA0AD8A4F1
:1030B00064D02550E90A09E02550EB0A03E12750C6
:1030C000900A03E00201006A03D00201010E006EC3
:1030D000005250E10101EF5306E1F05304E1F153D6
:1030E00002E1F25309E0EBC155F2ECC156F2EDC139
:1030F00057F2EEC158F238D0FF5307E102010053F6
:1031000004E1015302E102530AE00201FBC155F25E
:10311000FCC156F2FDC157F2FEC158F225D00F5343
:1031200006E1105304E1115302E1125309E00BC20E
:1031300055F20CC256F20DC257F20EC258F214D01C
:103140001F5306E1205304E1215302E1225309E019
:103150001BC255F21CC256F21DC257F21EC258F2D3
:1031600003D0010E006E12000201020102010401EF
:10317000836B03D00401010E836F0401846B04018F
:10318000835329E155C2E5F456C2E6F457C2E7F489
:1031900058C2E8F4250EE96F000EEA6F69EC33F0CF
:1031A00002012351550A07E12451AA0A04E1010E44
:1031B0000401836F10D004018451400A03E1010E21
:1031C000006E1200842B010E02015527000E5623BB
:1031D00057235823D4D7010E0401846F8351010A69
:1031E000D8A46DD1080E046E31C000F0000E016E3F
:1031F0000450040105E0003600900136FF0FF9D7B6
:103200000401305000108D6F01C08EF4000E8E133B
:103210008DC425F28EC426F232C033F2080E046E3D
:1032200034C000F0000E016E0450040105E00036C9
:1032300000900136FF0FF9D70401335000108B6F57
:1032400001C08CF4000E8C138BC44CF28CC44DF274
:1032500035C053F2080E046E3CC000F0000E016E43
:103260000450040105E0003600900136FF0FF9D745
:1032700004013B500010896F01C08AF4000E8A13CC
:1032800089C44EF28AC44FF235C000F0000E016EC0
:1032900089C404F08AC405F001EC3BF0000E026E14
:1032A000036E020155510026565101225751022248
:1032B0005851032204018B510024856F8C51012049
:1032C000866F000E0220876F000E0320886F85C472
:1032D00038F286C439F287C43AF288C43BF2080E49
:1032E000046E37C000F0000E016E0450040105E0CA
:1032F000003600900136FF0FF9D704013650001256
:10330000000E011200C050F201C051F2000E026E18
:10331000036E050E046E0450040107E000360090B1
:10332000013602360336FF0FF7D704018D51002412
:10333000086E8E510120096E000E02200A6E000EEA
:1033400003200B6E010E046E000E056E066E076EF6
:1033500008C000F009C001F00AC002F00BC003F081
:103360000450005E0550015A0650025A0750035A95
:103370008DC404F08EC405F0000E066E076E67EC77
:103380002BF00050040185250201346F0150040127
:1033900086210201356F0250040187210201366F38
:1033A0000350040188210201376F04018B5102018F
:1033B0005525006E04018C5102015621016E000E4C
:1033C0005721026E000E5821036E00C021F001C08B
:1033D00022F002C023F003C024F00401895100242C
:1033E0000201276F04018A5101200201286F000E9B
:1033F0000220296F000E03202A6F8DC42DF28EC487
:103400002EF22E332D332E9F3B503C1054E039507A
:10341000381005E038C07FF439C080F408D045C0CA
:103420007FF446C080F447C081F448C082F47FC472
:1034300000F080C401F081C402F082C403F00201F4
:103440003451005E3551015A3651025A3751035AF0
:1034500033C204F0000E056E066E076EE0EC1FF03E
:1034600000C07FF401C080F402C081F403C082F484
:10347000000E035C08E1000E025C05E10F0E015C2A
:1034800002E1F50E005C04E2010E0401846F12D02B
:103490000401000E825D08E1000E815D05E1FF0E72
:1034A000805D02E1F50E7F5D02E2846B03D00401D2
:1034B000010E846F04D00401010E006E120004019D
:1034C00084C400F012000001025006180E6E086A53
:1034D000096A0B6A0350076457EF1BF006500A6E27
:1034E000068E028E03500B6E0750036E000E0B64A7
:1034F000A7EF1AF00B50075ED8B448EF1BF0070E89
:10350000076416EF1BF0075E00C008F001C000F072
:1035100002C001F0026A074E48EF1BF00764EBEFB0
:103520001AF0075E00C008F001C000F0016A074E03
:1035300048EF1BF00764C9EF1AF0075E00C008F0FF
:10354000006A074E48EF1BF00764B0EF1AF00AC09C
:1035500002F005C001F004C000F0086A74EF1CF02E
:10356000030E0764BBEF1AF0075E08380F0B086EF6
:10357000074E48EF1BF0D8900832074E48EF1BF07B
:10358000D8900832074E48EF1BF0D890083248EF29
:103590001BF0030E0764DAEF1AF0075E08380F0B12
:1035A000086E0038F00B082600380F0B006E074E2F
:1035B00048EF1BF0D89000320832074E48EF1BF05E
:1035C000D89000320832074E48EF1BF0D8900032F6
:1035D000083248EF1BF0030E076402EF1BF0075E92
:1035E00008380F0B086E0038F00B082600380F0B58
:1035F000006E0138F00B002601380F0B016E074EEC
:1036000048EF1BF0D890013200320832074E48EFE5
:103610001BF0D890013200320832074E48EF1BF001
:10362000D89001320032083248EF1BF0030E0764D5
:1036300033EF1BF0075E08380F0B086E0038F00BF5
:10364000082600380F0B006E0138F00B00260138F9
:103650000F0B016E0238F00B012602380F0B026EC1
:10366000074E48EF1BF0D890023201320032083288
:10367000074E48EF1BF0D890023201320032083278
:10368000074E48EF1BF0D890023201320032083268
:10369000096A000E0EAE3CEF1CF0081E001E011E53
:1036A000021E082A0022012202223CEF1CF00750D1
:1036B000D8A45DEF1BF074EF1CF0096A02C00AF099
:1036C000028E068E0750035C076ED8B42FEF1CF0F5
:1036D000070E0764FDEF1BF0075E0450096E0550EE
:1036E000046E0650056E066A074E2FEF1CF0070E9B
:1036F0000764D2EF1BF0075E0450096E0550046E9C
:10370000056A074E2FEF1CF0070E0764B0EF1BF0A1
:10371000075E0450096E046A074E2FEF1CF0070E77
:10372000076497EF1BF00AC002F074EF1CF0030E61
:103730000764A2EF1BF0075E09380F0B096E074EF6
:103740002FEF1CF0D8900932074E2FEF1CF0D890C5
:103750000932074E2FEF1CF0D89009322FEF1CF0E2
:10376000030E0764C1EF1BF0075E09380F0B096EEB
:103770000438F00B092604380F0B046E074E2FEFA8
:103780001CF0D89004320932074E2FEF1CF0D8906D
:1037900004320932074E2FEF1CF0D8900432093260
:1037A0002FEF1CF0030E0764E9EF1BF0075E0938EA
:1037B0000F0B096E0438F00B092604380F0B046E4A
:1037C0000538F00B042605380F0B056E074E2FEF5A
:1037D0001CF0D890053204320932074E2FEF1CF04E
:1037E000D890053204320932074E2FEF1CF0D890E2
:1037F0000532043209322FEF1CF0030E07641AEF72
:103800001CF0075E09380F0B096E0438F00B09260F
:1038100004380F0B046E0538F00B042605380F0B27
:10382000056E0638F00B052606380F0B066E074EA0
:103830002FEF1CF0D8900632053204320932074EC1
:103840002FEF1CF0D8900632053204320932074EB1
:103850002FEF1CF0D8900632053204320932086A84
:10386000000E0EAE3CEF1CF0091E041E051E061EC7
:10387000092A0422052206220950082604500022A3
:1038800005500122065002220EBE53EF1CF0D8A0B4
:1038900062EF1CF00232013200320832033E62EF66
:1038A0001CF06EEF1CF0D8B068EF1CF0000E081E84
:1038B000001E011E021E082A0022012202220A7E88
:1038C00068EF1CF0010E0C6E16EC28F076EF1CF081
:1038D000020E0C6E16EC28F076EF1CF0040E0C6E47
:1038E00007EC3EF076EF1CF0000E0C6E12000401A7
:1038F0007F6B806B7F517C25E96E000E7D21EA6E27
:10390000EECF02F00250000A49E07F517C25E96EBB
:10391000000E7D21EA6EEECF02F002502E0A02E187
:103920007FC480F47F517C25E96E000E7D21EA6E14
:10393000EECFB7F4D0EC3DF00050011019E0840E4A
:10394000906F040E916F7F519027D8B0912B7F51CB
:103950007C25E96E000E7D21EA6EEECFB7F444ECD3
:103960003EF090C4E1FF91C4E2FF00C0E6FF13D037
:10397000840EE16E040EE26E04017F51E126D8B0A0
:10398000E22A7F517C25E96E000E7D21EA6EEECFA2
:1039900000F000C0E6FF04017F2BACD7840EE16E7F
:1039A000040EE26E7F51E126D8B0E22AE66A805327
:1039B00059E080C47FF4030E8025026E036A000E76
:1039C0000322800E006E800E0318005C02E102509C
:1039D0007F5D48E27F51010F006E016A000E0122F7
:1039E000840E0024E96E040E0120EA6EEECF02F090
:1039F0000250000A1DE1020E8025026E036A000ECD
:103A00000322800E0318006E800E005C02E17F51DD
:103A1000025C0CE3840EE16E040EE26E7F51E1263F
:103A2000D8B0E22A200EE66E7F2BE5D704011AD02B
:103A3000840EE16E040EE26E7F51E126D8B0E22AD8
:103A40007F51010F006E016A000E0122840E0024D6
:103A5000E96E040E0120EA6EEECF00F000C0E6FF32
:103A60007F2BA9D704017F070A0E7F5D2FE2840E0A
:103A7000E96E040EEA6E7F51E926D8B0EA2AEECF4D
:103A80008EF47F07840EE96E040EEA6E7F51E926FC
:103A9000D8B0EA2AEECF8DF47F07840EE96E040ECB
:103AA000EA6E7F51E926D8B0EA2AEECF8CF47F5136
:103AB00007080CE3840EE16E040EE26E7F51E126EE
:103AC000D8B0E22A200EE66E7F2BF1D78F6B020171
:103AD0003E6B3F6B3C6B3D6B38C2E5F439C2E6F49C
:103AE0003AC2E7F43BC2E8F4250E0401E96F000E88
:103AF000EA6F69EC33F00401816B826B806B020129
:103B00003F51261902E125513E191DE13E6B3F6BE5
:103B10003C4B3D2B3C5138250401E56F02013D51E2
:103B200039210401E66F000E02013A210401E76F1A
:103B3000000E02013B210401E86F250EE96F000E23
:103B4000EA6F69EC33F00401806B7F6B7F510A08E8
:103B500020E37F5102013E25006E000E3F21016EE1
:103B6000250E0024E96E000E0120EA6EEECF04F06F
:103B7000840EE96E040EEA6E04017F51E926D8B086
:103B8000EA2AEECF02F004500218D8B4802B7F2B23
:103B9000DDD7814B822B250E02013E25E96E000EFA
:103BA0003F21EA6EEECF83F4200E3E27000E3F2326
:103BB000040180510B0A11E082510201511903E105
:103BC000505104018119040102E11E0E806F0401AD
:103BD0008351000A02E1190E806F80510A088FE2BA
:103BE000140E805D49E2200E02013E5D006E000E63
:103BF0003F59016E00C03EF201C03FF21A0E00268E
:103C0000000E0122250E0024E96E000E0120EA6E4E
:103C1000EECF2BF2EECF2CF22AEC3BF01C0E3E2521
:103C2000006E000E3F21016E250E0024E96E000E8D
:103C30000120EA6EEECF44F2EECF45F2EECF46F22F
:103C4000EECF47F29FEC37F00E0E02013E25006EDC
:103C5000000E3F21016E250E0024E96E000E0120AA
:103C6000EA6EEECF5BF2EECF5CF2EECF59F2EECF22
:103C70005AF2010E006E120004017EAF0CD0840EC9
:103C8000B76F040EB86F7F0E7E15B96F0CEC29F07C
:103C9000010E006E1200006A12006E0E0401E05D5B
:103CA000D8A0D0D0640E046EE0C400F09DEC3DF0CE
:103CB000120E0026016A000E0122020E046E000E92
:103CC00001BEFF0E026E036E0450000107E00036D5
:103CD0000090013602360336FF0FF7D700012A0E97
:103CE00000267D0E0122000E022200C0F6FF01C058
:103CF000F7FF02C0F8FF0900F5CF00F00900F5CF8B
:103D000001F00900F5CF02F00900F5CF03F0000E35
:103D1000046E000E056E000E066E7E0E076E99ECA8
:103D20002EF000C0E1F401C0E2F402C0E3F403C0ED
:103D3000E4F4640E046EE0C400F09DEC3DF008C0B5
:103D400000F00A0E046E9DEC3DF0090E0026016A9B
:103D5000000E0122020E046E000E01BEFF0E026E66
:103D6000036E0450000107E0003600900136023671
:103D70000336FF0FF7D700012A0E00267D0E012221
:103D8000000E022200C0F6FF01C0F7FF02C0F8FFDC
:103D90000900F5CF00F00900F5CF01F00900F5CFDB
:103DA00002F00900F5CF03F0E1C404F0E2C405F02D
:103DB000E3C406F0E4C407F099EC2EF000C0E1F48F
:103DC00001C0E2F402C0E3F403C0E4F40A0E046E9E
:103DD000E0C400F09DEC3DF008C000F0020E046E5F
:103DE000000E016E026E036E0450000107E0003603
:103DF0000090013602360336FF0FF7D700012A0E76
:103E000000267D0E0122000E022200C0F6FF01C036
:103E1000F7FF02C0F8FF0900F5CF00F00900F5CF69
:103E200001F00900F5CF02F00900F5CF03F0E1C47D
:103E300004F0E2C405F0E3C406F0E4C407F099EC32
:103E40002EF012000401E0510A08D8B083D00A0E07
:103E5000046EE0C400F09DEC3DF0090E0026016AFE
:103E6000000E0122020E046E000E01BEFF0E026E55
:103E7000036E0450000107E0003600900136023660
:103E80000336FF0FF7D700012A0E00267D0E012210
:103E9000000E022200C0F6FF01C0F7FF02C0F8FFCB
:103EA0000900F5CF00F00900F5CF01F00900F5CFCA
:103EB00002F00900F5CF03F0000E046E000E056E4F
:103EC000000E066E7E0E076E99EC2EF000C0E1F437
:103ED00001C0E2F402C0E3F403C0E4F40A0E046E8D
:103EE000E0C400F09DEC3DF008C000F0020E046E4E
:103EF000000E016E026E036E0450000107E00036F2
:103F00000090013602360336FF0FF7D700012A0E64
:103F100000267D0E0122000E022200C0F6FF01C025
:103F2000F7FF02C0F8FF0900F5CF00F00900F5CF58
:103F300001F00900F5CF02F00900F5CF03F0E1C46C
:103F400004F0E2C405F0E3C406F0E4C407F099EC21
:103F50002EF012000001020E046EE0C400F0000E0C
:103F6000016E026E036E0450000107E000360090FF
:103F7000013602360336FF0FF7D72A0E00267D0ED4
:103F80000122000E022200C0F6FF01C0F7FF02C0AE
:103F9000F8FF0900F5CF00F00900F5CF01F00900A6
:103FA000F5CF02F00900F5CF03F0000E046E000E0D
:103FB000056E000E066E7E0E076E99EC2EF0120056
:103FC00000010B6A0A6A096A086A0E6A0334083635
:103FD0000450085E0550D8A0053C095E0650D8A0E4
:103FE000063C0A5E0750D8A0073C0B5EE86AD8A0E2
:103FF000010E0E5E0336070E0C6E033408360936CA
:104000000A360B360E36045003A01AEF20F0085E75
:104010000550D8A0053C095E0650D8A0063C0A5EB3
:104020000750D8A0073C0B5EE86AD8A0010E0E5ED0
:104030002BEF20F008260550D8B0053C0926065085
:10404000D8B0063C0A260750D8B0073C0B26E86AD1
:10405000D8B0010E0E2603360C2EFDEF1FF00234F1
:10406000083609360A360B360E36045003A04CEFDC
:1040700020F0085E0550D8A0053C095E0650D8A087
:10408000063C0A5E0750D8A0073C0B5EE86AD8A041
:10409000010E0E5E5DEF20F008260550D8B0053CFD
:1040A00009260650D8B0063C0A260750D8B0073C6F
:1040B0000B26E86AD8B0010E0E260236070E0C6EEB
:1040C0000234083609360A360B360E36045002A082
:1040D0007DEF20F0085E0550D8A0053C095E065033
:1040E000D8A0063C0A5E0750D8A0073C0B5EE86AE1
:1040F000D8A0010E0E5E8EEF20F008260550D8B035
:10410000053C09260650D8B0063C0A260750D8B010
:10411000073C0B26E86AD8B0010E0E2602360C2E9C
:1041200060EF20F00134083609360A360B360E36B9
:10413000045002A0AFEF20F0085E0550D8A0053C67
:10414000095E0650D8A0063C0A5E0750D8A0073C7E
:104150000B5EE86AD8A0010E0E5EC0EF20F00826C4
:104160000550D8B0053C09260650D8B0063C0A26B2
:104170000750D8B0073C0B26E86AD8B0010E0E26CF
:104180000136070E0C6E0134083609360A360B3636
:104190000E36045001A0E0EF20F0085E0550D8A0D4
:1041A000053C095E0650D8A0063C0A5E0750D8A020
:1041B000073C0B5EE86AD8A0010E0E5EF1EF20F01E
:1041C00008260550D8B0053C09260650D8B0063C54
:1041D0000A260750D8B0073C0B26E86AD8B0010E73
:1041E0000E2601360C2EC3EF20F0003408360936B7
:1041F0000A360B360E36045001A012EF21F0085E8D
:104200000550D8A0053C095E0650D8A0063C0A5EC1
:104210000750D8A0073C0B5EE86AD8A0010E0E5EDE
:1042200023EF21F008260550D8B0053C092606509A
:10423000D8B0063C0A260750D8B0073C0B26E86ADF
:10424000D8B0010E0E260036070E0C6E003408366C
:1042500009360A360B360E36045000A043EF21F023
:10426000085E0550D8A0053C095E0650D8A0063C63
:104270000A5E0750D8A0073C0B5EE86AD8A0010E82
:104280000E5E54EF21F008260550D8B0053C0926F3
:104290000650D8B0063C0A260750D8B0073C0B267B
:1042A000E86AD8B0010E0E2600360C2E26EF21F05B
:1042B00000B069EF21F0045008260550D8B0053C45
:1042C00009260650D8B0063C0A260750D8B0073C4D
:1042D0000B26120000010450085E0550D8A0053CD2
:1042E000095E0650D8A0063C0A5E0750D8A0073CDD
:1042F0000B5E0336070E0C6E0334083609360A3699
:104300000B36045003A094EF21F0085E0550D8A0AE
:10431000053C095E0650D8A0063C0A5E0750D8A0AE
:10432000073C0B5EA1EF21F008260550D8B0053CF4
:1043300009260650D8B0063C0A260750D8B0073CDC
:104340000B2603360C2E7CEF21F00234083609369A
:104350000A360B36045003A0BDEF21F0085E05506D
:10436000D8A0053C095E0650D8A0063C0A5E07505E
:10437000D8A0073C0B5ECAEF21F008260550D8B044
:10438000053C09260650D8B0063C0A260750D8B08E
:10439000073C0B260236070E0C6E0234083609362F
:1043A0000A360B36045002A0E5EF21F0085E0550F6
:1043B000D8A0053C095E0650D8A0063C0A5E07500E
:1043C000D8A0073C0B5EF2EF21F008260550D8B0CC
:1043D000053C09260650D8B0063C0A260750D8B03E
:1043E000073C0B2602360C2ECDEF21F001340836A7
:1043F00009360A360B36045002A00EEF22F0085E92
:104400000550D8A0053C095E0650D8A0063C0A5EBF
:104410000750D8A0073C0B5E1BEF22F00826055082
:10442000D8B0053C09260650D8B0063C0A260750ED
:10443000D8B0073C0B260136070E0C6E0134083647
:1044400009360A360B36045001A036EF22F0085E1A
:104450000550D8A0053C095E0650D8A0063C0A5E6F
:104460000750D8A0073C0B5E43EF22F0082605500A
:10447000D8B0053C09260650D8B0063C0A2607509D
:10448000D8B0073C0B2601360C2E1EEF22F000346C
:10449000083609360A360B36045001A05FEF22F0C9
:1044A000085E0550D8A0053C095E0650D8A0063C21
:1044B0000A5E0750D8A0073C0B5E6CEF22F008267E
:1044C0000550D8B0053C09260650D8B0063C0A264F
:1044D0000750D8B0073C0B260036070E0C6E003490
:1044E000083609360A360B36045000A087EF22F052
:1044F000085E0550D8A0053C095E0650D8A0063CD1
:104500000A5E0750D8A0073C0B5E94EF22F0082605
:104510000550D8B0053C09260650D8B0063C0A26FE
:104520000750D8B0073C0B2600360C2E6FEF22F058
:1045300000B0A9EF22F0045008260550D8B0053C81
:1045400009260650D8B0063C0A260750D8B0073CCA
:104550000B261200410E04015C6F550E5D6F540E68
:104560005E6F4F0E5F6F5F0E606F450E616F580E8E
:10457000626F450E636F540E646F580E656F540E74
:10458000666F676B810E7C6F0F0E7D6F030E7E6F03
:1045900028EC18F05C0E04017C6F040E7D6F010E98
:1045A0007E6F77EC1CF00052D8B400D1580E040195
:1045B0007C6F030E7D6FC3EC3BF003012B6B2C6B08
:1045C000800E006E800E2C19005C02E12B51140845
:1045D00013E35C0E04017C6F030E7D6F2BEC38F04F
:1045E0005D0E03012B25E16E030E2C21E26E5CC3F0
:1045F000E6FF2B4B2C2BE4D7F1EC38F05DC37DF3B9
:104600005EC37EF303017F6B7D0E04017C6F030E9E
:104610007D6FB6EC32F000C04EF301C04FF300C026
:104620007CF401C07DF4D5EC3AF000C07DF4840E3A
:104630007C6FAFEC3DF060C37DF361C37EF303019B
:104640007F6B7D0E04017C6F030E7D6FB6EC32F044
:1046500000C050F301C051F300C07CF401C07DF4F0
:10466000D5EC3AF000C07DF4820E7C6FAFEC3DF0EB
:1046700063C37DF364C37EF303017F6B7D0E04018E
:104680007C6F030E7D6FB6EC32F000C052F301C0B8
:1046900053F300C07CF401C07DF4D5EC3AF000C0C7
:1046A0007DF4860E7C6FAFEC3DF066C37DF367C38F
:1046B0007EF303017F6B7D0E04017C6F030E7D6F23
:1046C000B6EC32F000C054F301C055F300C07CF4E6
:1046D00001C07DF4D5EC3AF000C07DF4880E7C6F0B
:1046E000AFEC3DF069C37DF36AC37EF36BC37FF328
:1046F0006CC380F30301816B7D0E04017C6F030E9C
:104700007D6FB6EC32F0D00E005E070E015A00C08D
:1047100056F301C057F300C07CF401C07DF4D5EC22
:104720003AF000C07DF48C0E7C6FAFEC3DF06EC3B0
:104730007DF303017E6B7D0E04017C6F030E7D6FA4
:10474000B6EC32F000C0FDF3010E04017C6F000EE8
:104750007D6F00C07EF44AEC3DF0210E0B6EFF0E23
:104760000A6E0B2E01D003D00A2EFED7FAD7600EA8
:104770000A6E0A2EFED700000000020E04017C6FB4
:10478000000E7D6F70C37EF44AEC3DF0210E0B6E7F
:10479000FF0E0A6E0B2E01D003D00A2EFED7FAD7D9
:1047A000600E0A6E0A2EFED70000000012006DECAB
:1047B00039F00D0E0401466F0A0E476F470E486F21
:1047C000350E496F2D0E4A6F440E4B6F610E4C6FC4
:1047D000740E4D6F610E4E6F200E4F6F4C0E506F6A
:1047E0006F0E516F670E526F670E536F650E546FE9
:1047F000720E556F200E566F560E576F320E586F51
:104800002E0E596F300E5A6F5B6B400ED36ED38EE7
:10481000080E966E800E846E836A400E956EFF0EB3
:10482000926E7E6A7F6A070E936EFF0E816E930E04
:10483000946EFF0E826E8A8A1F0ECD6ECF6ACE6A8C
:10484000AF0ED56ED59ED76AD66AD00EF26EF18EB7
:10485000F70E7C6E9E908C988C86C30E0B6EFF0EAE
:104860000A6E0B2E01D003D00A2EFED7FAD74B0EBC
:104870000A6E0A2EFED700008C968C880C0EAF6E46
:10488000AC8439EC3EF0460E04017C6F040E7D6F63
:1048900028EC3CF065EC3CF0FFEC29F004015C6B8B
:1048A0005D6B5E6B010E5F6F1DEC3DF00400010E51
:1048B000D16E810EB76F0F0EB86F030EB96F7AEC21
:1048C00030F00052F6E18C988C86010ED16E0D6BA3
:1048D0000E6B0F6B106B020E7C6F000E7D6F5AEC2F
:1048E0003EF000C011F4AAEC22F00400020E040114
:1048F0007C6F000E7D6F5AEC3EF0040111510018E0
:1049000016E07C6B7D6BFF0E7E6F4AEC3DF0210E56
:104910000B6EFF0E0A6E0B2E01D003D00A2EFED7AF
:10492000FAD7600E0A6E0A2EFED7000000000400BF
:1049300007EC37F0810E04017C6F0F0E7D6F030EC4
:104940007E6F28EC18F0FE0E04017C6F030E7D6F65
:10495000A00E7E6F77EC1CF07D0E04015C6F030EE1
:104960005D6FFE0E5E6F030E5F6F78EC3BF0040030
:104970001EEC26F05CEC32F056C35CF457C35DF4D9
:1049800054C35EF452C35FF44EC360F450C361F489
:104990000401626BBDEC2CF01EEC26F07D0E0401D0
:1049A0007C6F030E7D6FA80E7E6F7E0E7F6F000EF4
:1049B000806F52EC3BF07D0E7C6F030E7D6FBAEC86
:1049C0003CF000C07EF401C07FF47D0E7C6F030ECE
:1049D0007D6F20EC27F0040054EC37F08C988C9617
:1049E0009D80010ED16E03008AEC3DF07FEC11F04A
:1049F0002DEC3EF0F8D7FFD71D5021240401E56FC0
:104A00001E502220E66F000E2320E76F000E2420A8
:104A1000E86F250EE96F000EEA6F69EC33F0250EA2
:104A20001F24006E000E2020016E00C0E9FF01C0AF
:104A3000EAFFEECFB8F4000E0401B96FBA6FBB6F96
:104A4000000EB96FBA6FBB6FEECFB9F41DC048F25C
:104A50001EC049F21FC04AF220C04BF200C0E1FF65
:104A600001C0E2FFB7C4E6FFB7C4E6FF1D50212432
:104A7000E56F1E502220E66F000E2320E76F000E28
:104A80002420E86F250EE96F000EEA6F2DEC2FF061
:104A90001D50020127250401E56F1E500201282147
:104AA0000401E66F000E020129210401E76F000EE8
:104AB00002012A210401E86F250EE96F000EEA6F5A
:104AC0002DEC2FF0000E006E0401BB1908E1005020
:104AD000BA1905E1FF0EB91902E1B851FF0AD8B4BD
:104AE000A4D0B8C4C0F4B9C4C1F4BAC4C2F4BBC43D
:104AF000C3F4C037C091C137C237C337C0C4B8F49C
:104B0000C1C4B9F4C2C4BAF4C3C4BBF425C204F02E
:104B100026C205F0000E066E076EC0C400F0C1C4C8
:104B200001F0C2C402F0C3C403F0E0EC1FF000C007
:104B3000BCF401C0BDF402C0BEF403C0BFF4BCC4E9
:104B40001DF0BDC41EF025C204F026C205F0000E03
:104B5000066E076EC0C400F0C1C401F0C2C402F00A
:104B6000C3C403F0E0EC1FF008C000F009C001F07E
:104B70000AC002F00BC003F000C01FF001C020F01B
:104B80000401BC512124E56FBD512220E66F000EC7
:104B90002320E76F000E2420E86F250EE96F000E3A
:104BA000EA6F69EC33F0250E1F24006E000E202002
:104BB000016E00C0E9FF01C0EAFFEECFB8F4EECF0E
:104BC000B9F400C0E1FF01C0E2FFE66AE66A1D50E9
:104BD00021240401E56F1E502220E66F000E2320E1
:104BE000E76F000E2420E86F250EE96F000EEA6FD4
:104BF0002DEC2FF01D50020127250401E56F1E50FA
:104C0000020128210401E66F000E0201292104019E
:104C1000E76F000E02012A210401E86F250EE96FFB
:104C2000000EEA6F2DEC2FF04DD748C21DF049C29F
:104C30001EF04AC21FF04BC220F012001D5021246A
:104C40000401E56F1E502220E66F000E2320E76F5F
:104C5000000E2420E86F250EE96F000EEA6F69EC64
:104C600033F0250E1F24E96E000E2020EA6EEECFF1
:104C70007CF4000E04017D6F7E6F7F6F000E7D6FF0
:104C80007E6F7F6FEECF7DF40401000E006E7F1902
:104C900008E100507E1905E1FF0E7D1902E17C510B
:104CA000FF0A6DE07CC484F47DC485F47EC486F480
:104CB0007FC487F48437849185378637873784C4E7
:104CC0007CF485C47DF486C47EF487C47FF425C259
:104CD00004F026C205F0000E066E076E84C400F0D4
:104CE00085C401F086C402F087C403F0E0EC1FF035
:104CF00000C080F401C081F402C082F403C083F4D8
:104D000080C41DF081C41EF025C204F026C205F047
:104D1000000E066E076E84C400F085C401F086C4E0
:104D200002F087C403F0E0EC1FF008C000F009C0F7
:104D300001F00AC002F00BC003F000C01FF001C078
:104D400020F0040180512124E56F81512220E66F7B
:104D5000000E2320E76F000E2420E86F250EE96F78
:104D6000000EEA6F69EC33F0250E1F24E96E000E89
:104D70002020EA6EEECF7CF4EECF7DF485D7D4EC24
:104D80003CF02AEC3BF033C200F0000E016E026EE4
:104D9000036E25C204F026C205F0000E066E076EF3
:104DA00010EC3AF000C004F001C005F002C006F0BB
:104DB00003C007F044C200F045C201F046C202F051
:104DC00047C203F0E0EC1FF008C000F009C001F09A
:104DD0000AC002F00BC003F025C204F026C205F0A1
:104DE000000E066E076EE0EC1FF000C052F200509D
:104DF00002012F27000E30233123322325C204F075
:104E000026C205F0000E066E076E44C200F045C2D1
:104E100001F046C202F047C203F0E0EC1FF008C008
:104E200000F009C001F00AC002F00BC003F000C09E
:104E300040F201C041F202C042F203C043F212004C
:104E40002FC2E5F430C2E6F431C2E7F432C2E8F42E
:104E5000250E0401E96F000EEA6F69EC33F00401DE
:104E6000806B816B7F51815D02E17E51805D5AE2F2
:104E7000250E02014025E16E000E4121E26E040183
:104E800080517C25E96E81517D21EA6EEECF00F0E4
:104E900000C0E6FF010E02014027000E412342231D
:104EA0004323000E006E431908E10050421905E14A
:104EB0002651411902E14051251930E12FC2E5F494
:104EC00030C2E6F431C2E7F432C2E8F4250E040140
:104ED000E96F000EEA6F2DEC2FF0010E02012F2773
:104EE000000E302331233223406B416B426B436B06
:104EF000522B5251331903E1526B40EC31F02FC267
:104F0000E5F430C2E6F431C2E7F432C2E8F4250E2B
:104F10000401E96F000EEA6F69EC33F00401804B85
:104F2000812BA0D704012FC2E5F430C2E6F431C2D0
:104F3000E7F432C2E8F4250EE96F000EEA6F2DECBB
:104F40002FF0040180510201442704018151020124
:104F50004523000E462347233C5138250401E56FC5
:104F600002013D5139210401E66F000E02013A2190
:104F70000401E76F000E02013B210401E86F250EDA
:104F8000E96F000EEA6F69EC33F00E0E02013E2568
:104F9000006E000E3F21016E250E0024E16E000E12
:104FA0000120E26E5BC2E6FF5CC2E6FF59C2E6FF8B
:104FB0005AC2E6FF59C2E6FF5AC2E6FFE66AE66A4F
:104FC0005BC2E6FF5CC2E6FF59C2E6FF5AC2E6FFDB
:104FD0001C0E3E25006E000E3F21016E250E0024A2
:104FE000E16E000E0120E26E44C2E6FF45C2E6FF1C
:104FF00046C2E6FF47C2E6FF3C5138250401E56F93
:1050000002013D5139210401E66F000E02013A21EF
:105010000401E76F000E02013B210401E86F250E39
:10502000E96F000EEA6F2DEC2FF0120000010CB0BA
:1050300059EF28F00CA201EF29F00E6A000E02646D
:1050400070EF28F0F00E0214D8A43BEF28F0023ADB
:1050500001380F0B02260138F00B016E00380F0BE0
:1050600001260038F00B006E08380F0B00260838B8
:10507000F00B086E0E84D89002BE54EF28F008366C
:105080000036013602360E2A02BE54EF28F00836EA
:105090000036013602360E2A02BE54EF28F00836DA
:1050A0000036013602360E2A0E500364F5EF28F062
:1050B000035E0BBC08AEFBEF28F0D880800E0864BE
:1050C0000030000E002201220222D8A0FBEF28F0BF
:1050D000023201320032034A01EF29F0FBEF28F0DF
:1050E00001C002F000C001F008C000F0086A000E24
:1050F0000E860264A7EF28F0F00E0214D8A48FEFFA
:1051000028F0023A01380F0B02260138F00B016E2D
:1051100000380F0B01260038F00B006E0E84D8907B
:1051200002BE54EF28F00036013602360E2A02BEC7
:1051300054EF28F00036013602360E2A02BE54EF34
:1051400028F00036013602360E2A54EF28F001C04E
:1051500002F000C001F0006A000E0E960E88026494
:10516000D4EF28F0F00E0214D8A4BFEF28F0023AD2
:1051700001380F0B02260138F00B016E0E84D89017
:1051800002BE54EF28F0013602360E2A02BE54EF5A
:1051900028F0013602360E2A02BE54EF28F00136FE
:1051A00002360E2A54EF28F001C002F0016A000E08
:1051B0000E86026407EF29F0F00E0214D8A4E3EF84
:1051C00028F0023A0E84D89002BE54EF28F002363E
:1051D0000E2A02BE54EF28F002360E2A02BE54EF09
:1051E00028F002360E2A54EF28F0010E0C6EDFEC88
:1051F0003DF00BEF29F0020E0C6E86EC3EF00BEF4B
:1052000029F0040E0C6E07EC3EF00BEF29F0080EAF
:105210000C6E64EC3EF0120002013E6B3F6B3C6B87
:105220003D6BA1EC31F0E7EC37F0D4EC3CF038C248
:10523000E5F439C2E6F43AC2E7F43BC2E8F4250EDD
:105240000401E96F000EEA6F69EC33F00401BB6BF7
:1052500002013F51261902E125513E191DE13E6B25
:105260003F6B3C4B3D2B3C5138250401E56F02015F
:105270003D5139210401E66F000E02013A2104017B
:10528000E76F000E02013B210401E86F250EE96F74
:10529000000EEA6F69EC33F0250E02013E25E96E3F
:1052A000000E3F21EA6EEECF02F00250E50A0BE05D
:1052B000250E3E25E96E000E3F21EA6EEECF02F08C
:1052C0000250000A03E1010E0401BB6F200E02012F
:1052D0003E27000E3F230401BB53BAE0BB51010A35
:1052E000D8A48AD0200E02013E5F000E3F5B04016D
:1052F000BA6BBA510A081AE3BA5102013E25006E90
:10530000000E3F21016E250E0024E16E000E0120EB
:10531000E26E0401BA51B725E96E000EB821EA6EBB
:10532000EECF00F000C0E6FFBA2BE3D71C0EBA6F39
:10533000200EBA5D11E2BA5102013E25006E000E48
:105340003F21016E250E0024E16E000E0120E26E69
:10535000E66A0401BA2BECD71A0E02013E25006E54
:10536000000E3F21016E250E0024E16E000E01208B
:10537000E26E2BC2E6FF2CC2E6FF0B0E3E25006E4E
:10538000000E3F21016E250E0024E16E000E01206B
:10539000E26EB9C4E6FF0D0E0401BA6FBA511908E6
:1053A00011E3BA5102013E25006E000E3F21016E4D
:1053B000250E0024E16E000E0120E26EE66A040173
:1053C000BA2BECD702013C5138250401E56F0201EC
:1053D0003D5139210401E66F000E02013A2104011A
:1053E000E76F000E02013B210401E86F250EE96F13
:1053F000000EEA6F2DEC2FF02AEC3BF012000301B7
:105400002B6B2C6B800E2C19006E800E005C02E161
:10541000280E2B5DD8B0ABD0046A8CB8042A010EDC
:105420000418006E000E00B0100E8C18100B8C1AB1
:105430002D51000A0CE1F80E8C1665EC35F000C019
:105440002EF301C02FF302C030F303C031F3030188
:105450002D51010A0BE18C8011EC35F000C032F3C4
:1054600001C033F302C034F303C035F303012D51FF
:10547000020A12E1F80E8C14006E00C08CFF020EBE
:1054800000108C6E0DEC36F000C036F301C037F31F
:1054900002C038F303C039F303012D51030A0CE1B4
:1054A000030E8C12B9EC35F000C03AF301C03BF3A7
:1054B00002C03CF303C03DF303012D51040A12E185
:1054C000F80E8C14006E00C08CFF040E00108C6E61
:1054D00015EC34F000C03EF301C03FF302C040F3CE
:1054E00003C041F303012D51050A0CE1050E8C1296
:1054F000BDEC34F000C042F301C043F302C044F3FA
:1055000003C045F303012D51060A12E1F80E8C1475
:10551000006E00C08CFF060E00108C6E69EC34F03B
:1055200000C046F301C047F302C048F303C049F38B
:1055300003012D51070A0CE1070E8C1261EC36F0C5
:1055400000C04AF301C04BF302C04CF303C04DF35B
:105550007AEC3EF003012D2B800E070A006E800EC0
:105560002D19005CD8A02D6B2B4B2C2B4BD7120088
:105570008C8603012B6B2C6B800E2C19006E800E19
:10558000005C02E1080E2B5DD8B09FD02D51000ABF
:105590000CE1F80E8C1665EC35F000C02EF301C05E
:1055A0002FF302C030F303C031F303012D51010A80
:1055B0000BE18C8011EC35F000C032F301C033F305
:1055C00002C034F303C035F303012D51020A12E186
:1055D000F80E8C14006E00C08CFF020E00108C6E52
:1055E0000DEC36F000C036F301C037F302C038F3DB
:1055F00003C039F303012D51030A0CE1030E8C1291
:10560000B9EC35F000C03AF301C03BF302C03CF303
:1056100003C03DF303012D51040A12E1F80E8C146E
:10562000006E00C08CFF040E00108C6E15EC34F080
:1056300000C03EF301C03FF302C040F303C041F39A
:1056400003012D51050A0CE1050E8C12BDEC34F05E
:1056500000C042F301C043F302C044F303C045F36A
:1056600003012D51060A12E1F80E8C14006E00C0E1
:105670008CFF060E00108C6E69EC34F000C046F30F
:1056800001C047F302C048F303C049F303012D51A1
:10569000070A0CE1070E8C1261EC36F000C04AF3E9
:1056A00001C04BF302C04CF303C04DF37AEC3EF063
:1056B00003012D2B800E070A006E800E2D19005C51
:1056C000D8A02D6B2B4B2C2B57D78C96120000019A
:1056D0000C6A07BE0C2A0D6A0B6A0A6A096A086A14
:1056E0000350021001100010D8B40BEF2CF003503F
:1056F00007180E6E0EBE0D1E07AE8AEF2BF0041EAD
:10570000051E061E071E042AD8B4052AD8B4062A88
:10571000D8B4072A03AE98EF2BF0001E011E021E1C
:10572000031E002AD8B4012AD8B4022AD8B4032A06
:10573000035007100E6E0EBEBEEF2BF06AEC21F088
:105740000CBEDFEF2BF00DAE0BEF2CF0001E011E98
:10575000021E031E002AD8B4012AD8B4022AD8B4E3
:10576000032A081E091E0A1E0B1E082AD8B4092A7D
:10577000D8B40A2AD8B40B2A0BEF2CF007AED8EF16
:105780002BF003BED2EF2BF003500B6E02500A6ECB
:105790000150096E0050086E036A026A016A006ACD
:1057A000A3EF2BF0036A026A016A006A002A000C68
:1057B000031E021E011E001E0C8E9EEF2BF0082AF7
:1057C000D8B4092AD8B40A2AD8B40B2A0450085CE1
:1057D000D8A4A3EF2BF00550095CD8A4A3EF2BF0BD
:1057E00006500A5CD8A4A3EF2BF007500B5CD8A49A
:1057F000A3EF2BF00B6A0A6A096A086A002AD8B478
:10580000012AD8B4022AD8B4032A03AEA3EF2BF09E
:105810000E6A0E88FF0C0E6A0CA011EF2CF014EC2F
:105820003EF0000F12000001086A096A0750D8B460
:10583000AAEF2CF00350D8B4AFEF2CF002500618AA
:105840000A6E028E068E0E6A02C008F001C00CF0CD
:1058500000C00DF004500D5E0550D8A0053C0C5E54
:105860000650D8A0063C085E086A0C6A0D6AD8A0EB
:1058700041EF2CF0D8900232013200320832010E92
:105880000E6E0750035ED8A04EEF2CF07E0E0E2455
:105890000326D8B0B4EF2CF054EF2CF07E0E0E247B
:1058A0000326D8A0B9EF2CF0180E0B6E0D360C366F
:1058B00008360036013602360E360450005E0550BA
:1058C000D8A0053C015E0650D8A0063C025E063416
:1058D0000E120EA06FEF2CF00D807AEF2CF004501A
:1058E00000260550D8B0053C01260650D8B0062841
:1058F00002260D900B2E56EF2CF0A0EF2CF0D89036
:105900000036013602360E360450005E0550D8A02F
:10591000053C015E0650D8A0063C025E06340E101F
:10592000010B0D26D8B00C2AD8B4082AD8A4A0EFB1
:105930002CF008320C320D32032AD8B4B4EF2CF01C
:105940000AAE089E0850026E0C50016E0D50006E9B
:10595000BCEF2CF0010E90EC3EF0BCEF2CF0020EF0
:1059600064EC3EF0BCEF2CF0040E07EC3EF0BCEF14
:105970002CF0080EDFEC3DF01200BC0E04015C5D63
:10598000006E070E5D59016E00C05CF401C05DF44D
:105990007F0E00145C6F01C05DF4000E5D170F0EEA
:1059A0005E15006E00C05EF4005202E1010E5E6FF3
:1059B0005F511F0803E3010E5F5D02E2010E5F6F9E
:1059C00060511708D8A0606B61513B08D8A0616B8B
:1059D00062513B08D8A0626B62C408F00832089E8E
:1059E00008C062F4090E006E5CC406F05DC407F0E6
:1059F0000050040105E0063606900736FF0FF9D780
:105A0000040106C059F207C05AF25EC404F0000E49
:105A1000056E050E026E04C000F005C001F00250D4
:105A2000040105E0003600900136FF0FF9D70401AC
:105A3000065000120750011200C059F201C05AF27C
:105A40005F5100100201596F01C05AF2000E5A1343
:105A500060C402F0000E036E0B0E006E02C006F072
:105A600003C007F00050020105E006360690073635
:105A7000FF0FF9D7020106C05BF207C05CF261C4F8
:105A800004F0000E056E050E026E04C000F005C0A5
:105A900001F00250020105E0003600900136FF0FD0
:105AA000F9D70201065000120750011200C05BF244
:105AB00001C05CF2085000105B6F01C05CF2000E88
:105AC0005C13120000010B6A0C6A0A6A086A035030
:105AD000D8B4EBEF2DF0028E9E0E035E03BE76EF80
:105AE0002DF0D8B476EF2DF0DBEF2DF0036C080E1F
:105AF000035CD8A0A8EF2DF0036E083600C008F0B4
:105B000001C000F002C001F0026A080E035CD8A0D8
:105B1000A8EF2DF0036E083600C008F001C000F0B9
:105B2000016A080E035CD8A0A8EF2DF0036E0836BA
:105B300000C008F0006A080E035CD8A0A8EF2DF0A2
:105B4000036E0836086A0350D8A4D890B4EF2DF03D
:105B50000350D8B4B4EF2DF0D890023201320032A5
:105B60000832032EACEF2DF00BBC08A0C5EF2DF0D2
:105B7000D8A0C5EF2DF0082AD8B4002AD8B4012A3D
:105B8000D8B4022A02BEEFEF2DF00AAEEBEF2DF0F3
:105B9000021E011E001E081E082AD8B4002AD8B40E
:105BA000012AD8B4022AEBEF2DF0026A016A006ADA
:105BB000086AEBEF2DF00B800BAEF5EF2DF0026ACB
:105BC0000AAEF5EF2DF0026E016E006E086E0A3619
:105BD0000232F5EF2DF0000E0C6AF6EF2DF0010EFB
:105BE0000C6EC1EC3DF0F6EF2DF0FF0E0250036E8F
:105BF0000150026E0050016E0850006E120000014C
:105C00000B6A0C6A086A0350D8B484EF2EF002C005
:105C10000AF0028E9E0E035E03AE74EF2EF0036C4C
:105C2000080E035CD8A041EF2EF0036E083600C0CA
:105C300008F001C000F002C001F0026A080E035C27
:105C4000D8A041EF2EF0036E083600C008F001C066
:105C500000F0016A080E035CD8A041EF2EF0036E3D
:105C6000083600C008F0006A080E035CD8A041EFB7
:105C70002EF0036E0836086A0350D8A4D8904DEF72
:105C80002EF00350D8B44DEF2EF0D89002320132EE
:105C900000320832032E45EF2EF00BBC08A05EEF59
:105CA0002EF0D8A05EEF2EF0082AD8B4002AD8B47F
:105CB000012AD8B4022A02BE88EF2EF00AAE84EF81
:105CC0002EF0021E011E001E081E082AD8B4002A4B
:105CD000D8B4012AD8B4022A84EF2EF0026A016AED
:105CE000006A086A84EF2EF00B800BAE8FEF2EF067
:105CF000026A0AAE8FEF2EF0026E016E006E086E21
:105D00000A3602328FEF2EF00C6A000E90EF2EF062
:105D1000010E0C6E000EC1EC3DF090EF2EF0FF0E68
:105D20000250036E0150026E0050016E0850006E6A
:105D300012000001086A096A000E076203641FEF7F
:105D40002FF0025006180A6E075003267E0ED8A0C8
:105D5000B0EF2EF0035ED8B024EF2FF0B4EF2EF0AA
:105D6000035ED8A029EF2FF0028E068E02C00EF03F
:105D700001C00BF000C00DF000500402F4CF0CF095
:105D800001500502F4CF00F0F3CF08F00402F35005
:105D90000C26F4500822000E00220D500502F3508C
:105DA0000C26F4500822000E002202500402F35088
:105DB0000826F450002202500502016A000E01225A
:105DC000F3500026F45001220D500602F35008262D
:105DD000F4500022026A000E012202220B50060239
:105DE000F3500026F4500122000E02220E5006024B
:105DF000F3500126F450022202BE07EF2FF00836BE
:105E00000036013602360306D8B429EF2FF01AEF18
:105E10002FF0D880800E08640030000E002201228E
:105E20000222D8A01AEF2FF0023201320032034AC8
:105E300024EF2FF00AAE029E000E2CEF2FF0010E81
:105E400064EC3EF02CEF2FF0020E07EC3EF02CEF4E
:105E50002FF0040EDFEC3DF012006CEC3EF0090E6A
:105E6000006EE5C4F0F4E6C4F1F4E7C4F2F4E8C46B
:105E7000F3F4005008E00401F037F091F137F23705
:105E8000F337FF0FF7D70401180EEF6FFF0EF46F13
:105E9000B0EC38F0005205E021EC3EF0010E006E4F
:105EA0001200FF0E0401F86F73EC3EF0FF0E0401C8
:105EB000F86F73EC3EF0FE0E0401F86F73EC3EF0E9
:105EC0000401EB6BEC6BEC51010802E1EB51FF08B4
:105ED0000EE3EB51E925E96EEC51EA21EA6EEECFD3
:105EE000F8F473EC3EF00401EB4BEC2BECD704011F
:105EF000FF0EF86F73EC3EF0FF0E0401F86F73ECC9
:105F00003EF0FF0E0401F86F73EC3EF000C0EBF4BE
:105F1000000E0401EC6F1F0EEB15016EECC402F0D5
:105F2000000E021601C0EBF402C0ECF4000E0218E1
:105F300002E1050E011805E021EC3EF0020E006EB4
:105F40001200FF0E0401F86F73EC3EF00050FF0AE0
:105F5000F8E121EC3EF0006A120000010A6A0350E9
:105F6000D8A40A800750D8A40A820A50D8B411EFE6
:105F700030F0030AD8B4CAEF2FF00AB0C5EF2FF003
:105F800006AE0FEF30F00DEF30F002AE0DEF30F057
:105F90000FEF30F00250800B0A6E029E0650800B0D
:105FA000069E0A18D8B4DBEF2FF00A50D8B40DEFD4
:105FB00030F00FEF30F00750035CD8B4E5EF2FF06E
:105FC000D8A001EF30F007EF30F00650025CD8B4F3
:105FD000EFEF2FF0D8A001EF30F007EF30F00550D1
:105FE000015CD8B4F9EF2FF0D8A001EF30F007EF43
:105FF00030F00450005CD8B411EF30F0D8B007EFA7
:1060000030F00A52D8B40FEF30F00DEF30F00A52F2
:10601000D8B40DEF30F00FEF30F0D8801200D890E8
:106020001200D880D8841200120000010D6A096A9B
:10603000086A01500010D8B4000C015005180A6E0F
:106040000ABE0D1E0B6A05AE2BEF30F0041E051EB6
:10605000042AD8B4052A01AE33EF30F0001E011E29
:10606000002AD8B4012A015005100A6E0ABE4BEF6F
:1060700030F076EC3AF00BB062EF30F00DAE000C81
:10608000001E011E002AD8B4012A081E091E082A73
:10609000D8B4092A000C05AE5DEF30F001BE59EF0F
:1060A00030F00150096E0050086E016A006A3EEF40
:1060B00030F0016A006A002A000C011E001E0B2A43
:1060C00039EF30F0082AD8B4092A0450085CD8A463
:1060D0003EEF30F00550095CD8A43EEF30F0096A7D
:1060E000086A002AD8B4012A01AE3EEF30F0000061
:1060F000FF0C1200B9C400F0010E016E005004E064
:1061000001360190FF0FFBD701C01CF0011C006E8F
:1061100000C01BF0090E0401B725196E000EB8214E
:106120001A6E19C0E9FF1AC0EAFF0150EF12090EFA
:106130001924E96E0050EF16BB6B0A0EBB5D07E237
:10614000FF0EF86F73EC3EF00401BB2BF6D76CEC3E
:106150003EF00401EF6BF06BF16BF26BF36B950E9D
:10616000F46FB0EC38F000C0BBF421EC3EF0040159
:10617000BB51010A03E0010E006E1200BB6BFF0E63
:10618000BB5D19E26CEC3EF0010E0401EF6FF06BA9
:10619000F16BF26BF36BFF0EF46FB0EC38F000C0F4
:1061A000BAF421EC3EF00401BA51000A02E1006A9F
:1061B0001200BB2BE4D7010E006E12000401E16B4C
:1061C000E26BE36BE46B839AE06B200EE05D29E207
:1061D000E1C405F0E2C406F0E3C407F0E4C408F04B
:1061E0000536059006360736083605C0E1F406C0C8
:1061F000E2F407C0E3F408C0E4F4838E046A83BCCD
:10620000042A04500510E16F06C0E2F407C0E3F46D
:1062100008C0E4F4000EE213E313E413839EE02BC2
:10622000D4D7838AE4A905D0006A016A026A036AA6
:106230001200FF0EE115056EFF0EE215066EFF0E51
:10624000E315076E1F0EE415086E05C0E1F406C0E5
:10625000E2F407C0E3F408C0E4F406C000F007C0AD
:1062600001F008C002F0000E08BEFF0E036E00C071
:10627000E1F401C0E2F402C0E3F403C0E4F412006C
:106280001DC048F21EC049F21FC04AF220C04BF2A6
:10629000A1EC31F0E7EC37F0D4EC3CF002014851CE
:1062A00021240401E56F0201495122200401E66F17
:1062B000000E2320E76F000E2420E86F250EE96F03
:1062C000000EEA6F69EC33F0250E02014A25E16EFB
:1062D000000E4B21E26E2BC2E6FF2CC2E6FF4851B6
:1062E00021240401E56F0201495122200401E66FD7
:1062F000000E2320E76F000E2420E86F250EE96FC3
:10630000000EEA6F2DEC2FF0020148512725040101
:10631000E56F0201495128210401E66F000E0201D8
:1063200029210401E76F000E02012A210401E86F10
:10633000250EE96F000EEA6F2DEC2FF02AEC3BF0F2
:1063400012000401E06B1D6A1E6A040E1F6E000E2F
:10635000206E21C0E5F422C0E6F423C0E7F424C097
:10636000E8F4250EE96F000EEA6F69EC33F0205077
:106370000201261902E125511F1817E11F6A206A40
:106380001D4A1E2A1D5021240401E56F1E502220A3
:10639000E66F000E2320E76F000E2420E86F250E25
:1063A000E96F000EEA6F69EC33F0250E1F24E96EE9
:1063B000000E2020EA6EEECF02F00250000A14E137
:1063C000010E1F24006E000E2020016E250E0024F9
:1063D000E96E000E0120EA6EEECF02F00250000AD4
:1063E00003E1010E0401E06F0401020E1F26000EFE
:1063F0002022E053BCE0E06B020E1F5E000E205A2C
:10640000120000010D6A086A0050D8B4000C04188C
:106410000A6E0ABE0D1E0B6A04AE11EF32F0041EA6
:10642000042A00A016EF32F0001E002A00500410CB
:106430000A6E0ABE3DEF32F00450085E00360034AA
:106440000836045008260036060E0C6E0034083656
:10645000045000B0085E00A0082600360C2E26EF7F
:1064600032F000A008260BB04FEF32F00DAE000C5A
:10647000001E002A081E082A000C04AE4BEF32F062
:1064800000BE48EF32F00050086E006A36EF32F07E
:10649000006A002A000C001E0B2A1CEF32F0082AAA
:1064A0000450085CD8A436EF32F0086A002A00AE27
:1064B00036EF32F0FF0C1200850E0401B76FFAECD4
:1064C0003DF000C0B7F4000E0401B86F9EEC3CF044
:1064D00000C04EF3000E03014F6F830E0401B76F2F
:1064E000FAEC3DF000C0B7F4000E0401B86F9EEC6A
:1064F0003CF000C050F3000E0301516F870E040101
:10650000B76FFAEC3DF000C0B7F4000E0401B86FAD
:106510009EEC3CF000C052F3000E0301536F890E55
:106520000401B76FFAEC3DF000C0B7F4000E0401AF
:10653000B86F9EEC3CF000C054F3000E0301556FA1
:106540008D0E0401B76FFAEC3DF000C0B7F4000EF9
:106550000401B86F9EEC3CF000C056F3000E03013E
:10656000576FD00E5627070E572312007CC4E9FF41
:106570007DC4EAFFEECF02F002C07EF40250200A92
:1065800004E004017E51090A04E104017C4B7D2BE7
:10659000EDD77F6B806B816B7E512D0A04E1812BDF
:1065A0007C4B7D2B05D07E512B0A02E17C4B7D2B51
:1065B0007CC4E9FF7DC4EAFFEECF00F000C07EF4AA
:1065C00000C0E0F4EDEC3DF000521AE07FC400F0B2
:1065D00080C401F00A0E046E000E056EDCEC39F08A
:1065E000300E04017E5D026E036A000E035A0250F3
:1065F00000247F6F03500120806F7C4B7D2BD8D708
:106600000401815308E07F510008006E80C401F04E
:10661000E86A015612007FC400F080C401F0120045
:1066200003010051000A08E10401B76B9EEC3BF046
:1066300000C003F301C004F303010051010A09E1A2
:10664000010E0401B76F9EEC3BF000C005F301C0E2
:1066500006F303010051020A09E1020E0401B76FBB
:106660009EEC3BF000C007F301C008F303010051AA
:10667000030A09E1030E0401B76F9EEC3BF000C072
:1066800009F301C00AF30301002B800E030A006E18
:10669000800E0019005CD8A0006B0B6B0C6B0D6BAF
:1066A0000E6B0F6B106B010E8114006E04E0010E77
:1066B0000B6F000E0C6F81A204D0010E0D6F000E47
:1066C0000E6F030181A404D0010E0F6F000E106F36
:1066D00012006CEC3EF0090E006EE5C4F0F4E6C466
:1066E000F1F4E7C4F2F4E8C4F3F4005008E0040164
:1066F000F037F091F137F237F337FF0FF7D7040196
:10670000110EEF6FFF0EF46FB0EC38F0005205E0A1
:1067100021EC3EF0010E006E1200FF0E0401F86F36
:1067200073EC3EF00050FE0AF8E10401EB6BEC6BF9
:10673000020EEC5D02E1000EEB5D14E2EB51E92587
:10674000ED6FEC51EA21EE6FFF0EF86F73EC3EF047
:10675000EDC4E1FFEEC4E2FF00C0E6FF0401EB4B35
:10676000EC2BE6D70401FF0EF86F73EC3EF0FF0E42
:106770000401F86F73EC3EF021EC3EF0006A120069
:106780001BC317F31CC318F31DC319F31EC31AF35D
:106790001FC31BF320C31CF321C31DF322C31EF32D
:1067A00023C31FF324C320F325C321F326C322F3FD
:1067B00027C323F328C324F329C325F32AC326F3CD
:1067C00013C327F314C328F3000E0301296F2A6FA4
:1067D00023512725006E24512821016E255129219E
:1067E000026E26512A21036E1F51002620510122DC
:1067F00021510222225103221B5100261C51012249
:106800001D5102221E510322175100261851012248
:10681000195102221A510322140E046E000E056E45
:10682000066E076EE0EC1FF01200B1C2ADF2B2C20C
:10683000AEF2B3C2AFF2B4C2B0F2B5C2B1F2B6C2F8
:10684000B2F2B7C2B3F2B8C2B4F2B9C2B5F2BAC2C8
:10685000B6F2BBC2B7F2BCC2B8F2BDC2B9F2BEC298
:10686000BAF2BFC2BBF2C0C2BCF2DEEC30F000C074
:10687000BDF201C0BEF202C0BFF203C0C0F202010D
:10688000B9510026BA510122BB510222BC51032248
:10689000B5510026B6510122B7510222B851032248
:1068A000B1510026B2510122B3510222B451032248
:1068B000AD510026AE510122AF510222B051032248
:1068C000050E046E000E056E066E076EE0EC1FF0FE
:1068D0001200D9C2D5F2DAC2D6F2DBC2D7F2DCC2DC
:1068E000D8F2DDC2D9F2DEC2DAF2DFC2DBF2E0C2F8
:1068F000DCF2E1C2DDF2E2C2DEF2E3C2DFF2E4C2C8
:10690000E0F2E5C2E1F2E6C2E2F2E7C2E3F2E8C297
:10691000E4F2DEEC30F000C0E5F201C0E6F202C0C5
:10692000E7F203C0E8F20201E1510026E251012240
:10693000E3510222E4510322DD510026DE510122FF
:10694000DF510222E0510322D9510026DA510122FF
:10695000DB510222DC510322D5510026D6510122FF
:10696000D7510222D8510322050E046E000E056E87
:10697000066E076EE0EC1FF01200C5C2C1F2C6C27F
:10698000C2F2C7C2C3F2C8C2C4F2C9C2C5F2CAC207
:10699000C6F2CBC2C7F2CCC2C8F2CDC2C9F2CEC2D7
:1069A000CAF2CFC2CBF2D0C2CCF2D1C2CDF2D2C2A7
:1069B000CEF2D3C2CFF2D4C2D0F2DEEC30F000C0BF
:1069C000D1F201C0D2F202C0D3F203C0D4F202016C
:1069D000CD510026CE510122CF510222D0510322A7
:1069E000C9510026CA510122CB510222CC510322A7
:1069F000C5510026C6510122C7510222C8510322A7
:106A0000C1510026C2510122C3510222C4510322A6
:106A1000050E046E000E056E066E076EE0EC1FF0AC
:106A2000120075C271F276C272F277C273F278C246
:106A300074F279C275F27AC276F27BC277F27CC2C6
:106A400078F27DC279F27EC27AF27FC27BF280C296
:106A50007CF281C27DF282C27EF283C27FF284C266
:106A600080F2DEEC30F000C081F201C082F202C0A0
:106A700083F203C084F202017D5100267E5101227F
:106A80007F51022280510322795100267A5101223E
:106A90007B5102227C51032275510026765101223E
:106AA000775102227851032271510026725101223E
:106AB0007351022274510322050E046E000E056EFE
:106AC000066E076EE0EC1FF0120061C25DF262C25A
:106AD0005EF263C25FF264C260F265C261F266C2D6
:106AE00062F267C263F268C264F269C265F26AC2A6
:106AF00066F26BC267F26CC268F26DC269F26EC276
:106B00006AF26FC26BF270C26CF2DEEC30F000C061
:106B10006DF201C06EF202C06FF203C070F20201AA
:106B2000695100266A5101226B5102226C510322E5
:106B300065510026665101226751022268510322E5
:106B400061510026625101226351022264510322E5
:106B50005D5100265E5101225F51022260510322E5
:106B6000050E046E000E056E066E076EE0EC1FF05B
:106B700012009DC299F29EC29AF29FC29BF2A0C2DD
:106B80009CF2A1C29DF2A2C29EF2A3C29FF2A4C235
:106B9000A0F2A5C2A1F2A6C2A2F2A7C2A3F2A8C205
:106BA000A4F2A9C2A5F2AAC2A6F2ABC2A7F2ACC2D5
:106BB000A8F2DEEC30F000C0A9F201C0AAF202C0D7
:106BC000ABF203C0ACF20201A5510026A65101228E
:106BD000A7510222A8510322A1510026A25101224D
:106BE000A3510222A45103229D5100269E5101224D
:106BF0009F510222A0510322995100269A5101224D
:106C00009B5102229C510322050E046E000E056E5C
:106C1000066E076EE0EC1FF0120089C285F28AC290
:106C200086F28BC287F28CC288F28DC289F28EC244
:106C30008AF28FC28BF290C28CF291C28DF292C214
:106C40008EF293C28FF294C290F295C291F296C2E4
:106C500092F297C293F298C294F2DEEC30F000C048
:106C600095F201C096F202C097F203C098F20201B9
:106C700091510026925101229351022294510322F4
:106C80008D5100268E5101228F51022290510322F4
:106C9000895100268A5101228B5102228C510322F4
:106CA00085510026865101228751022288510322F4
:106CB000050E046E000E056E066E076EE0EC1FF00A
:106CC0001200EDC2E9F2EEC2EAF2EFC2EBF2F0C25C
:106CD000ECF2F1C2EDF2F2C2EEF2F3C2EFF2F4C264
:106CE000F0F2F5C2F1F2F6C2F2F2F7C2F3F2F8C234
:106CF000F4F2F9C2F5F2FAC2F6F2FBC2F7F2FCC204
:106D0000F8F2DEEC30F000C0F9F201C0FAF202C095
:106D1000FBF203C0FCF20201F5510026F6510122FC
:106D2000F7510222F8510322F1510026F2510122BB
:106D3000F3510222F4510322ED510026EE510122BB
:106D4000EF510222F0510322E9510026EA510122BB
:106D5000EB510222EC510322050E046E000E056E6B
:106D6000066E076EE0EC1FF012001D502124040196
:106D7000E56F1E502220E66F000E2320E76F000E05
:106D80002420E86F250EE96F000EEA6F69EC33F0FE
:106D9000250E1F24E96E000E2020EA6EEECFB7F418
:106DA000EECFB8F40401B851FF0A02E1FF0EB719A3
:106DB0002DE02DC204F02EC205F0B7C400F0B8C417
:106DC00001F047EC3CF000C01DF001C01EF02DC2E8
:106DD00004F02EC205F0B7C400F0B8C401F047ECCF
:106DE0003CF008C000F009C001F000C01FF001C075
:106DF00020F000C01FF001C020F01F361F90203689
:106E0000B7C42BF2B8C42CF22AEC3BF01200020EED
:106E100004017C6F000E7D6F5AEC3EF000C0FEF363
:106E20000050FF0A03E1580E0301FE6F04017C6B62
:106E30007D6B5AEC3EF000C00AF40050010F0401D3
:106E40000A6F7C6B7D6B0AC47EF44AEC3DF0640EE5
:106E5000046E0AC400F09DEC3DF0300E00240401E5
:106E6000036F640E046E0AC400F09DEC3DF008C090
:106E700000F000C05CF45CC40AF40A0E046E5CC44A
:106E800000F09DEC3DF0300E00240401046F0A0E6A
:106E9000046E5CC400F09DEC3DF008C000F0300EC4
:106EA00000240401056F1200010E04017C6F000E26
:106EB0007D6F5AEC3EF000C0FDF329D00C0E0301AB
:106EC000016F000E026F3AD03C0E016F000E026F90
:106ED00035D0B40E016F000E026F30D02C0E016F52
:106EE000010E026F2BD0580E016F020E026F26D0DA
:106EF000080E016F070E026F21D0100E016F0E0EEB
:106F0000026F1CD00C0E016F000E026F17D0030130
:106F1000FD51000AD3E0FD51010AD6E0FD51020AFD
:106F2000D8E0FD51030ADAE0FD51040ADCE0FD512E
:106F3000050ADEE0FD51060AE0E0E4D712002BC2AC
:106F400004F02CC205F0000E066E076E04C0B7F404
:106F500005C0B8F406C0B9F407C0BAF40401B737E5
:106F6000B791B837B937BA3725C204F026C205F051
:106F7000000E066E076EB7C400F0B8C401F0B9C4C5
:106F800002F0BAC403F0E0EC1FF000C01DF001C035
:106F90001EF025C204F026C205F0000E066E076E34
:106FA000B7C400F0B8C401F0B9C402F0BAC403F029
:106FB000E0EC1FF008C000F009C001F00AC002F0C8
:106FC0000BC003F000C01FF001C020F01200250E1E
:106FD0001F24E16E000E2020E26EFF0EE66E010E11
:106FE0001F24006E000E2020016E250E0024E16E8D
:106FF000000E0120E26EFF0EE66E1D5021240401FA
:10700000E56F1E502220E66F000E2320E76F000E72
:107010002420E86F250EE96F000EEA6F2DEC2FF0AB
:107020001D50020127250401E56F1E500201282191
:107030000401E66F000E020129210401E76F000E32
:1070400002012A210401E86F250EE96F000EEA6FA4
:107050002DEC2FF01200250E02014025E96E000EE6
:107060004121EA6EEECF00F07CC4E1FF7DC4E2FF77
:1070700000C0E6FF010E4027000E412342234323B8
:10708000000E006E431908E10050421905E1265137
:10709000411902E14051251920E1010E2F27000E70
:1070A000302331233223406B416B426B436B522BB5
:1070B0005251331903E1526BB5EC36F02FC2E5F4AF
:1070C00030C2E6F431C2E7F432C2E8F4250E04011E
:1070D000E96F000EEA6F69EC33F012000201386BC1
:1070E000396B3A6B3B6B3C6B3D6B3E6B3F6B406B64
:1070F000416B426B436B2B6B2C6B2F6B306B316B8B
:10710000326B446B456B466B476B216A226A236A7C
:10711000246A276B286B296B2A6B1D6A1E6A486BD1
:10712000496B1F6A206A4A6B4B6B256B266B2D6B74
:107130002E6B4C6B4D6B4E6B4F6B506B516B346BBE
:10714000356B366B376B336B526B536B546B556BC4
:10715000566B576B586B596B5A6B5B6B5C6B1200C1
:10716000400E0401EF25F86F73EC3EF0F3C4F8F421
:1071700073EC3EF0F2C4F8F473EC3EF0F1C4F8F4B2
:1071800073EC3EF0F0C4F8F473EC3EF0F4C4F8F4A1
:1071900073EC3EF0FF0E0401F86F73EC3EF000C09C
:1071A000F5F40401F66BF76B0401F551000A16E0E3
:1071B000F551010A13E0F6C401F0F7C402F0F64BF2
:1071C000F72B4E0E025C02E1200E015C07E2FF0E7F
:1071D000F86F73EC3EF000C0F5F4E6D7F5C400F0AC
:1071E000120002013C51382504017C6F02013D511F
:1071F000392104017D6F000E02013A2104017E6FE6
:10720000000E02013B2104017F6FB76BFCEC24F000
:107210007CC4E5F47DC4E6F47EC4E7F47FC4E8F4FE
:10722000250E0401E96F000EEA6F69EC33F0250EBC
:1072300002013E25E16E000E3F21E26EE50EE66E94
:107240007CC4E5F47DC4E6F47EC4E7F47FC4E8F4CE
:10725000250E0401E96F000EEA6F2DEC2FF01200ED
:1072600000010C6A0E6A0250D8A44AEF39F001C03E
:1072700002F000C001F0006A0E860250D8A44AEF66
:1072800039F001C002F0016A0E960E880250D8B49F
:107290005CEF39F00E50035ED8A4D8A062EF39F04D
:1072A000D89002BE68EF39F0003601360236032E60
:1072B00051EF39F062EF39F0010E0C6E64EC3EF0E4
:1072C0006CEF39F0020E0C6EDFEC3DF06CEF39F034
:1072D000040E0C6E86EC3EF01200780E0301FE6F79
:1072E000440EFF6F410E0401006F540E016F410EFA
:1072F000026F780E036F780E046F780E056F430EE1
:10730000066F530E076F560E086F096B000E0201D1
:10731000FD6F000EFE6F000E03012D6F000E006F5B
:10732000000E0201FF6F000E156E000E166E000EAD
:10733000176E000E186E000E0301116F000E126F13
:10734000000E136F000E146F12000301115333E08F
:107350008C888C96410E0B6EFF0E0A6E0B2E01D0A0
:1073600003D00A2EFED7FAD7C30E0A6E0A2EFED716
:1073700000008C98410E0B6EFF0E0A6E0B2E01D092
:1073800003D00A2EFED7FAD7C30E0A6E0A2EFED7F6
:1073900000008C888C96410E0B6EFF0E0A6E0B2E31
:1073A00001D003D00A2EFED7FAD7C30E0A6E0A2EDA
:1073B000FED700008C981200000100500402F4CFA8
:1073C00009F0F3CF08F001500502F4CF0BF0F3CF32
:1073D0000AF000500502F3500926F4500A22E86A28
:1073E0000B2201500402F3500926F4500A22E86AE5
:1073F0000B2205AE00EF3AF000500A5C01500B582A
:1074000001AE07EF3AF004500A5C05500B5808C073
:1074100000F009C001F00AC002F00BC003F0120036
:1074200000010D6A03AE20EF3AF0001E011E021E9D
:10743000031E000E002A012202220322810E0D26C5
:1074400007AE2DEF3AF0041E051E061E071E000EA5
:10745000042A0522062207220D2AA7EC3AF00DA0E5
:1074600043EF3AF0001E011E021E031E081E091EF5
:107470000A1E0B1E000E002A0122022203220822ED
:1074800009220A220B221200030E0401B76F9EECA0
:107490003BF034EC3DF03E0E046E050E056E420EE0
:1074A000066E800E076E99EC2EF0330E046E330ECE
:1074B000056E530E066E760E076E99EC2EF0000EDA
:1074C000046E000E056E000E066E810E076EADECAA
:1074D0002FF0010ED8B0000E006E005204E0010E35
:1074E0000301116F02D00301116B1200000101347E
:1074F000083609360450085E0550D8A0053C095EE0
:10750000003601360F0E0C6E013408360936045071
:1075100000A092EF3AF0085E0550D8A0053C095E45
:1075200097EF3AF008260550D8B0053C09260036FA
:1075300001360C2E84EF3AF000B0A5EF3AF004507B
:1075400008260550D8B0053C0926000012000001AD
:10755000220E0C6E086A096A0A6A0B6A0C06D8B415
:10756000D4EF3AF0D8900B320A32093208320332A3
:10757000023201320032D8A0AEEF3AF00C06D8B495
:10758000CCEF3AF0045008260550092206500A2292
:1075900007500B22B3EF3AF0045008260550092299
:1075A00006500A2207500B2212000A0E046E000E2B
:1075B000056E7CC400F07DC401F015EC30F008C00D
:1075C00000F009C001F000C07EF401C07FF40A0E93
:1075D000046E000E056E7CC400F07DC401F015EC55
:1075E00030F0040E036E00C002F00350000104E00E
:1075F00002360290FF0FFAD7025004017E11006E8E
:10760000120000010B6A0A6A096A00500402F4CFF2
:1076100009F0F3CF08F001500502F4CF0BF0F3CFDF
:107620000AF000500502F3500926F4500A22E86AD5
:107630000B2201500402F3500926F4500A22E86A92
:107640000B2208C000F009C001F00AC002F00BC014
:1076500003F01200020E02012B5D046E000E2C5985
:10766000056E33C200F0000E016E026E036E000E56
:10767000066E076E10EC3AF000C02FF201C030F237
:1076800002C031F203C032F20201345100242F6FE4
:1076900035510120306F36510220316F37510320B0
:1076A000326F1200810E0401B56F040EB66F7CC4F8
:1076B000B7F47DC4B8F47EC4B9F47FC4BAF480C40E
:1076C000BBF4B50EBC6F040EBD6F3AEC00F000C009
:1076D000B3F401C0B4F4005004017C25E16E015004
:1076E0007D21E26EE66AB3C400F0B4C401F012007A
:1076F0005CC460F45DC461F460C402F061C403F072
:107700000401604B612B5EC4E9FF5FC4EAFF5E4B7E
:107710005F2BEECF00F002C0E1FF03C0E2FF00C02C
:10772000E6FF02C0E9FF03C0EAFFEECF00F000521F
:10773000E3E15CC400F05DC401F01200C26A070E10
:10774000C012C08EB7C400F0003600900036009022
:107750000050C212C28080EC3EF0C282C2B2FED79C
:10776000080E026EC4CF00F0000E016E025005E05C
:10777000003600900136FF0FFAD7C3500012000EFA
:107780000112C29012000201406B416B426B436BCD
:107790007CC4E1FF7DC4E2FF44C2E6FF45C2E6FFD0
:1077A00046C2E6FF47C2E6FF526B2FC2E5F430C285
:1077B000E6F431C2E7F432C2E8F4250E0401E96FC1
:1077C000000EEA6F69EC33F01200000100C008F00F
:1077D0000150006E016A026A036A0B6A0C6A016A50
:1077E000026A036A960E036E0A6A00AEFEEF3BF071
:1077F000081E001E082AD8B4002A0A8E00C001F014
:1078000008C000F0086A026A30EC39F01200010E7C
:1078100003011219006E00C012F3005202E0D58E6F
:1078200016D0D59ED6CF13F3000E146FD7CF15F315
:10783000000E166F15C301F0006A00C015F301C0F9
:1078400016F30050131301501413D76AD66A1200AE
:1078500004017E6B7E517C25E96E000E7D21EA6E6F
:10786000EECF02F00250000A0DE07E517C25E96E59
:10787000000E7D21EA6EEECFB7F44FEC3EF004012E
:107880007E2BE8D77CC400F07DC401F0120000011B
:10789000086A096A100E0C6E013408360936045065
:1078A000085E0550D8A0053C095ED8B05FEF3CF0FB
:1078B000045008260550D8B0053C0926D89000365B
:1078C00001360C2E4CEF3CF01200819A82948E0E01
:1078D00004017C6F7D6BAFEC3DF0900E04017C6F7A
:1078E000AA0E7D6FAFEC3DF0810E0401B76FFAEC8C
:1078F0003DF07F0E001404017D6F800E7C6FAFECB5
:107900003DF0120093980401E26B080EE25D15E26F
:10791000010EE015006EE1C401F0000E01160050EA
:10792000011003E0818896EF3CF08198819A818A6A
:10793000E133E033E19FE22BE8D712000F0E0401A0
:10794000B715B96F040E026EB7C400F0B8C401F0E9
:107950000250040107E001320032019E01BC018E99
:10796000FF0FF7D704010A0E0002F3CF00F0B95160
:10797000002612007CC47EF47DC47FF47EC4E9FF3F
:107980007FC4EAFF04017E4B7F2BEECF00F0005254
:10799000F5E17C517E5D006E7D517F59016E010ED7
:1079A000005E000E015A12001DC000F01EC001F062
:1079B0002DC204F02EC205F001EC3BF01FC002F016
:1079C00020C003F003320232039E02500024020161
:1079D0002B6F035001202C6F120000010350071879
:1079E000D8A402EF3DF002500618D8A402EF3DF0F3
:1079F00001500518D8A402EF3DF000500418D8B487
:107A0000D8841200D89412001200040E0201FD2541
:107A1000016E000EFE21026E01C0FDF202C0FEF2F8
:107A200003010251025C02E10151015C05E3020124
:107A3000FD6BFE6B010EFF6F1200949A9496948872
:107A4000C66A04015C51C6125E51C6125D51C7126E
:107A50005E5305E05F51000AD8B4C78C03D05F5372
:107A6000D8A4C78CC68A120000010050086E0150CD
:107A7000006E016A026A036A0B6A0C6A960E036E54
:107A80000A6A00C001F008C000F0086A026A30EC1F
:107A900039F01200A6A202D00000FCD7A69C7DC43B
:107AA000AAFF7CC4A9FF7EC4A8FFA69EA684F29E5E
:107AB000550EA76EAA0EA76EA682F28EA69412008D
:107AC0000401E16B9388E06B070EE05D0CE2818AB4
:107AD000819A81A802D0E18F02D07F0EE117E133B5
:107AE000E19FE02BF1D7E1C400F01200000100504B
:107AF000086E0150006E0250016E0350026E036A60
:107B00000B6A0C6A9E0E036E0A6A020E0C6E16EC6D
:107B100028F0120005EC3DF010EC33F044EC3AF0A4
:107B2000A5EC39F007EC3CF0C0EC33F000C00BF4EE
:107B300001C00CF4B8EC2AF012000001086B080E2A
:107B40000C6E003408360450085ED8B0AAEF3DF041
:107B50000826D89000360C2EA1EF3DF01200819A35
:107B600082847CC4E0F4000E0401E16F82EC3CF0FE
:107B70007DC4E0F4000E0401E16F82EC3CF08294DD
:107B8000120000010B800BAECEEF3DF0026A0AAE90
:107B9000FF0E026E016E006E0A360232FF0E1200F8
:107BA0000401B7517A0807E3610EB75D04E3010EE3
:107BB000006EDCEF3DF0006A000E016E1200000165
:107BC0000B840BAEEBEF3DF0010E036E026A016A0F
:107BD000006A0A360232FF0E12000401E051390831
:107BE00007E3300EE05D04E3010E006EF9EF3DF0B7
:107BF000006A1200819A8284B7C4E0F4000E040186
:107C0000E16F82EC3CF060EC3DF0829412000001E8
:107C10000B820BAE12EF3EF0036802680168006849
:107C20000A360232FF0E120000010B1E0A1E091E48
:107C3000081E082AD8B4092AD8B40A2AD8B40B2AAC
:107C4000120019C0E9FF1AC0EAFF1C50EF12FF0E24
:107C50000401F86F73EC3EF01200810E0401B76F5F
:107C60000F0EB86F030EB96F7AEC30F00052F5E1E9
:107C70001200AC8A900EAB6E948E949C9EAA03D098
:107C8000AECF60F4FBD712000401B7517A0804E3C9
:107C9000610EB75DD8B0B79BB7C400F01200016A9F
:107CA000ACB2012A0150000A02E10000F8D7B7C4C3
:107CB000ADFF1200A69C7DC4AAFF7CC4A9FFA69EAE
:107CC000A680A8CF00F012000001026A016A006AD3
:107CD000086A036A000E120019C0E9FF1AC0EAFF21
:107CE0001B50EF161200F8C4C9FFC7A0FED7C9CFBA
:107CF00000F01200839E839A83BCFED7838A120011
:107D0000030E0A6E0A2EFED70000120000010AAE12
:107D1000029E000E12000001067E63EC1AF01200B3
:107D200000010B6A0B86FF0E12000000007FCDCC15
:107D30004C7B0AD723786F12037517B75171ACC506
:107D4000276EBD37066B95BF566777CC2B645F7087
:107D50000961FFE65B5D08E53C3C6042221B0000D8
:107D6000007F000020820000488500007A880040E3
:107D70001C8C0050438F002474928096189620BC6F
:107D80003E99286B6E9CF90215A0EC782DC1CAF2C1
:107D900049E2010000000A00000064000000E8035E
:107DA000000010270000A086010040420F008096CE
:107DB000980000E1F50500CA9A3B010000001000A0
:107DC00000000001000000100000000001000000A1
:107DD0001000000000010000001001000000080079
:107DE00000004000000000020000001000000080C1
:107DF000000000000400000020000000000100005E
:107E000000080000004000000000303132333435FB
:107E10003637383941424344454600FF303132332A
:107E200034353637383961626364656600FF0D0AA0
:107E3000256C642C25642F25642F25642C25303275
:107E4000643A253032642C25302E36662C25302EAF
:107E500036662C25302E36662C25302E36662C259F
:107E6000302E36662C25302E36662C25302E366682
:107E70002C25302E36662C25302E366600FF2C251C
:107E8000302E33662C25302E33662C25302E33666B
:107E90002C25302E33662C25752C25752C25752C1C
:107EA000256C642C256400FF0D0A53616D706C65B0
:107EB0002C446174652C54696D652C467261634471
:107EC00061792C4348312C4348322C4348332C43AE
:107ED00048342C4348352C4348362C4348372C43F0
:107EE00048382C56312C56322C56332C564241549D
:107EF000542C535441545553312C535441545553DD
:107F0000322C535441545553332C50554C53452C1B
:107F10004652455155454E435900FFFFFFFFFFFFB5
:020000040020DA
:020000040030CA
:0E00000000C81F16008781000FC00FE00F40E0
:0200000400F00A
:00000001FF
